:020000040800F2
:1000000080160020450100080D990008DB880008D3
:10001000A9950008F30D0008F5B6000800000000DF
:100020000000000000000000000000009D9A000891
:100030005934000800000000D999000839A90008C7
:100040005F0100085F0100085F0100085F01000810
:100050005F010008559A00085F0100085F01000871
:100060005F0100085F0100085F0100085F010008F0
:10007000AD330008BD330008CD330008DD33000880
:10008000ED330008FD3300085F0100085F01000840
:100090005F0100085F0100085F0100085F010008C0
:1000A0005F0100085F0100085F0100085F010008B0
:1000B0005F0100085F0100085F0100085F010008A0
:1000C0005F0100085F0100085F0100085F01000890
:1000D0005F010008BDB40008D1B40008E5B4000811
:1000E0005F0100085F0100085F0100085F01000870
:1000F00061AB00085F0100085F0100085F010008B4
:100100005F0100085F0100085F0100085F0100084F
:1001100085B000085F0100085F0100085F0100086A
:100120005F0100085F0100080D3400081D3400085D
:10013000DFF80CD000F0FEFA004800478DBF000841
:10014000801600200648804706480047FEE7FEE785
:10015000FEE7FEE7FEE7FEE7FEE7FEE7FEE7FEE777
:1001600009AB000831010008202A04DB203A21FAFB
:1001700002F00021704721FA02F3D040C2F12002C0
:10018000914008431946704740EA01039B0703D09A
:1001900009E008C9121F08C0042AFAD203E011F8C6
:1001A000013B00F8013B521EF9D27047D2B201E088
:1001B00000F8012B491EFBD270470022F6E710B56C
:1001C00013460A4604461946FFF7F0FF204610BDC5
:1001D000F0B480EA0102D40F4200B2EB410F02D228
:1001E0000246084611464A0042D0C30DDDB2C1F3B3
:1001F000C752AD1A202D35DAC1F3160141F40002C1
:1002000004B15242C5F1200602FA06F12A41104417
:10021000B3EBD05F23D0C4B1012DA0EBC35009DCF8
:10022000F0BC4FF0004202EAC352DBB200F500001E
:1002300000F0F5B9400000F1807000EBC350A0F170
:10024000807040EAD170490009E0490841EAC07174
:10025000A0EBC35000F50000400800EBC350F0BC19
:1002600000F0D4B96142012202EB4101001BF6E724
:10027000F0BC704781F00041AAE780F00040A7E79A
:1002800080EA010210B502F00043400022D04A008B
:100290001FD0010E01EB1261C0F35600C2F35602EB
:1002A00040F4000042F40002A0FB022000047F3969
:1002B000140400D0401C50EA124001D44000491EF2
:1002C000C2B20C0604EBD010401C4008802A02D0B9
:1002D00003E0002010BD20F00100002900DA00201A
:1002E000184310BD30B480EA010202F0004530F03E
:1002F000004221F0004013D090B1C30DD40DC2F3E1
:100300001601C0F31600E41A41F4000140F40002A3
:100310007D34914201D3641C00E04900002C02DAD4
:1003200030BC002070474FF400000023914201D3FD
:10033000891A034340084FEA4101F7D151B1914274
:1003400002D14FF0004105E002D24FF0010101E07F
:100350006FF0010103EBC450284430BC00F056B9E3
:100360002DE9F04D81EA030404F0004B21F0004533
:1003700014464FF0000A23F0004150EA050220D055
:1003800054EA01021DD0C5F30A570246C5F3130310
:10039000C1F31300C1F30A5640F4801543F48013EF
:1003A000A7EB0608101BD64608F2FD3873EB0500D4
:1003B00002D308F1010801E092185B41B8F1000F87
:1003C00003DA00200146BDE8F08D00204FF48011D3
:1003D000064684460EE0171B73EB050705D3121B78
:1003E00063EB050306434CEA010C49084FEA300071
:1003F00092185B4150EA0107EDD152EA030012D096
:1004000082EA040083EA0501084305D0101BAB41D2
:1004100006D20122002306E000224FF0004302E052
:100420006FF0010253101AEB06004CEB085110EB71
:100430000A0041EB0B01BDE8F04D00F01EB9C10F01
:1004400080EAE0700844CA079623002100F0E7B86C
:1004500096230022114600F0E2B80EB5C10F80EAE3
:10046000E0700844CA07002140F233438DE80E00D3
:100470000A460B4600F010F903B000BD00F0004240
:1004800020F00040C10DC0F3160040F400007F29A9
:1004900001DA00207047962903DCC1F19601C840BB
:1004A00001E096398840002AF4D04042704720F09D
:1004B0000040C10DC0F3160040F400007F2901DAAE
:1004C00000207047962903DCC1F19601C8407047AF
:1004D00096398840704700F0004230F000400AD062
:1004E000C10D01F56071C0F3160042EA0151C20866
:1004F00040071143704700200146704730B5041E85
:1005000071F1000404DB4FF00044404264EB010150
:10051000141E73F1000405DB1C464FF000435242E9
:1005200063EB0403994208BF904230BD01F00043E1
:1005300030B421F0004150EA010206D00A0DA2F5C4
:100540006072C1F31301002A02DC30BC0020704746
:10055000440F44EAC104C100E01830BC00EBC250B3
:1005600000F054B8002801DBC0F10040002901DB95
:10057000C1F1004181427047002801DBC0F1004019
:10058000002901DBC1F10041884270472DE9F05F8D
:100590000546002092469B468846064681464024F2
:1005A0001BE02846414647462246FFF7DDFD5346FD
:1005B0005A46C01A914110D311461846224600F0FF
:1005C00016F82D1A67EB01084F462246012000213C
:1005D00000F00DF817EB00094E41201EA4F10104B4
:1005E000DFDC484631462A464346BDE8F09F202AD4
:1005F00004DB203A00FA02F1002070479140C2F17A
:10060000200320FA03F31943904070470029A8BF44
:100610007047401C490008BF20F00100704710B42B
:10062000B0FA80FC00FA0CF050EA010404BF10BCE0
:10063000704749B1CCF1200421FA04F411FA0CF10D
:1006400018BF012121430843A3EB0C01CB1D4FEA46
:1006500000614FEA102042BF002010BC704700EB41
:10066000C35010440029A4BF10BC7047401C49006F
:1006700008BF20F0010010BC704710B5141E73F1C4
:10068000000408DA401C41F1000192185B411A4352
:1006900001D120F0010010BD2DE9F04D92469B469E
:1006A00011B1B1FA81F202E0B0FA80F22032904644
:1006B000FFF79DFF04460F4640EA0A0041EA0B019E
:1006C00053465A46084313D0114653EA010019D045
:1006D000C8F140025046FFF747FD05460E4650461A
:1006E00059464246FFF783FF084305D0012004E046
:1006F00020463946BDE8F08D0020054346EAE07605
:100700002C4337430A986305E40AA0EB0800002253
:10071000FD0A44EA47540A3002D500200146E9E7C1
:10072000010510196941DDE9084500196941BDE875
:10073000F04DA2E7064C074D06E0E06840F00103EB
:1007400094E8070098471034AC42F6D3FFF7F4FC66
:100750002CCA00084CCA000810B54A78052392FB41
:10076000F3F403FB14230A1D22F813004A78521CE9
:100770004A7010BD10B50346114840894FF6FF740A
:10078000A04201D0002010BD0E4840894FF6FF74F2
:10079000A04212D101200B4C60812046C380002072
:1007A0002081E081A081204601624262C06A007817
:1007B000401EE46A20700120E5E70020E3E7000026
:1007C000EC0D00206C0D002070B5044600200129BE
:1007D00006D002291DD0032934D0042964D14AE06F
:1007E0003F4D6D894FF6FF76B54211D101253C4E44
:1007F00075813546EC8000253581F581B58135461A
:100800002A626B62ED6A2D786D1EF66A35700120E2
:1008100063E0344D6D894FF6FF76B54211D1012565
:10082000304E75813546EC8000253581F581B581E6
:1008300035462A626B62ED6A2D786D1EF66A357058
:1008400002204AE0284D6D894FF6FF76B54211D15E
:100850000125254E75813546EC8000253581F581D1
:10086000B58135462A626B62ED6A2D786D1EF66A97
:100870003570032031E01D4D6D894FF6FF76B5428E
:1008800011D10125194E75813546EC800025358141
:10089000F581B58135462A626B62ED6A2D786D1E51
:1008A000F66A3570042018E00D4D6D894FF6FF761D
:1008B000B54211D101250A4E75813546EC800025DF
:1008C0003581F581B58135462A626B62ED6A2D78F6
:1008D0006D1EF66A3570012000BF00BF70BD0000BC
:1008E0006C0D0020AC0D0020EC0D00202C0E002023
:1008F00010B503460D4840894FF6FF74A04212D14F
:1009000001200A4C60812046C38000202081E081C4
:10091000A081204601624262C06A0078401EE46AFB
:100920002070022010BD0020FCE70000AC0D00206C
:1009300038B504461B4801F043F8AA20194981F84C
:100940003C001021174880F83D10002180F83E102F
:10095000082180F83F10002180F84010012180F824
:100960004110022180F84210002180F8431080F8E5
:10097000444009213C3009F0C3FF00909DF801106C
:10098000084880F845109DF8001080F846100B20AC
:100990000449C8800846C2883C31034807F016FF66
:1009A00038BD000022050020EC06002070B504468A
:1009B0006089B0F5967F7AD008DC012811D0022832
:1009C0001DD0642845D0C82867D151E1B0F5C87F53
:1009D0007ED0A0F57F40F03800287AD00F28F3D1E0
:1009E00022E0F948006800F4800010B10220608124
:1009F00004E048F225012046E26B9047F7E1F34816
:100A0000407800B1F3E1206A012805D0206A02286D
:100A100002D0206A032806D1642060810020E061B2
:100A2000A061206A6062E2E1E848407800B1DEE15E
:100A3000206A012805D0206A022802D0206A0328F3
:100A400006D1642060810020E061A061206A6062BC
:100A5000CDE1DE48407800B1C9E1DB48006800F430
:100A6000800028B948F225012046E26B9047BEE19C
:100A7000606A012804D0022808D0032813D10DE0B1
:100A800009F09EFC4FF4967060810CE009F07EFC4A
:100A90004FF4C870608106E009E0A1E109F076FC3E
:100AA000C820608100BF00BF002060619FE1C8488E
:100AB000B0F8400000F4807090B3C54890F8400052
:100AC00000F0300008B32046A16B88472C2001E0DD
:100AD00033E071E1BF49C870BF4880680068BE4913
:100AE00049680860BC4989680868BC49FFF7C8FBC9
:100AF0000546FFF7C3FCB849C968086001232C22EA
:100B00000821B44802F088FE16E064206081E069A4
:100B1000082811D948F221012046E26B90470BE0EA
:100B2000FFE76069401C60616069282804D948F2C9
:100B300026012046E26B904759E1A548B0F84000F5
:100B400000F48070002871D0A14890F8400000F0B7
:100B50000C00F8B1A048806800689F4949680860A7
:100B60009D49896808689D49FFF78AFB0546FFF79C
:100B700085FC9949C96808609748C068012310211D
:100B80000268944802F048FE4FF6FF706081002032
:100B9000E06165E08E4890F8400000F00100F8B197
:100BA0004FF6FF7060810020E0618B48806800682C
:100BB0008949496808608849896808688749FFF752
:100BC0005FFB0546FFF75AFC8349C9680860824805
:100BD000C0680123102102687E4802F01DFE3FE03C
:100BE0007B4890F8400000F0020000B34FF6FF7021
:100BF00060810020E0617848806800687649496833
:100C000008607549896808687449FFF739FB05462B
:100C1000FFF734FC7049C96808606F48C068012359
:100C2000102102686B4802F0F7FD19E00DE0642026
:100C30006081E069401CE061E069082810D948F251
:100C400021012046E26B90470AE06069401C606128
:100C50006069282804D948F226012046E26B9047B3
:100C6000D4E90810884202D04FF6FF706081BEE0E0
:100C70005748B0F8400000F4807000287AD05448FB
:100C800090F8400000F00C00E0B153488068006824
:100C90005149496808605049896808684F49FFF719
:100CA000EFFA0546FFF7EAFB4B49C96808604A4876
:100CB000C068012310210268464802F0ADFD002003
:100CC000E06163E0424890F8400000F0010028B382
:100CD0004148806800684049496808603E49896821
:100CE00008683E49FFF7CCFA0546FFF7C7FB3A49CB
:100CF000C96808603848C068012310210268354877
:100D000002F08AFDE069401CE061E06908283DD9F5
:100D100048F224012046E26B904737E02C4890F8D7
:100D2000400000F0020030B32B48806800682A4978
:100D3000496808602849896808682849FFF7A0FAC7
:100D40000546FFF79BFB2449C96808602248C06834
:100D50000123102102681F4802F05EFDE069401C7B
:100D6000E061E069082811D948F223012046E26BCE
:100D700090470BE00DE0E069401CE061E069082865
:100D800004D948F221012046E26B9047642060813B
:100D90000AE06069401C60616069282804D948F253
:100DA00026012046E26B9047D4E90810884202D021
:100DB0004FF6FF7060811AE04FF6FF7060810020EF
:100DC0002062606213E000000C000020900500200B
:100DD0006A0F0020BC0900200C0A002000401C46BD
:100DE0004FF6FF70608100202062606200BF00BF8C
:100DF00070BD00BFFEE730B50346002409E0188847
:100E00000D88A84201D0012030BD9B1C891C601CAC
:100E1000C4B29442F3DB0020F6E7F0B506460C4678
:100E2000022C14DDA01E81B2304609F069FD074690
:100E3000A01E355C4FF6FF7000EA0525601E305C91
:100E40000543BD4201D1012502E0002500E0002557
:100E5000E8B2F0BD10B5044604F4000030B1002241
:100E60004FF48051044806F0AFF804E0012211036A
:100E7000014806F0A9F810BD0018014010B504465D
:100E800004F4807030B100224FF48071044806F001
:100E90009BF804E001221102014806F095F810BD0C
:100EA0000008014010B5044604F4001028B10022E7
:100EB0000821054806F088F804E0012208210248CC
:100EC00006F082F810BD00000014014010B5044681
:100ED00004F4801028B100220421054806F074F8BB
:100EE00004E001220421024806F06EF810BD000063
:100EF0000018014010B5044604F4800030B100220F
:100F00004FF40041044806F05FF804E00122D103E9
:100F1000014806F059F810BD0018014010B504460C
:100F200004F4004030B100224FF48071044806F010
:100F30004BF804E001221102014806F045F810BD0B
:100F40000014014010B5044604F4804028B100228A
:100F50001021054806F038F804E00122102102486B
:100F600006F032F810BD00000018014010B504462C
:100F700004F4006030B100224FF48071044806F0A0
:100F800023F804E001221102014806F01DF810BD0B
:100F9000000C014010B5044604F4003030B10022CA
:100FA0004FF48071044806F00FF804E001221102AA
:100FB000014806F009F810BD0018014010B50446BC
:100FC00004F4803030B100224FF48061044805F011
:100FD000FBFF04E001229102014805F0F5FF10BD7E
:100FE0000018014010B5044604F0807028B10022BA
:100FF0000121054805F0E8FF04E0012211460248FE
:1010000005F0E2FF10BD00000010014010B50446DD
:1010100004F0007028B100224021054805F0D4FFFB
:1010200004E001224021024805F0CEFF10BD00007F
:101030000018014010B5044604F4007028B10022E5
:101040000221054805F0C0FF04E001220221024808
:1010500005F0BAFF10BD00000014014010B50446B1
:1010600004F4806028B100222021054805F0ACFF7F
:1010700004E001222021024805F0A6FF10BD000077
:101080000014014010B5044604F4006030B10022A1
:101090004FF48071044805F097FF04E0012211022B
:1010A000014805F091FF10BD000C014010B5044649
:1010B00004F4005028B100228021054805F084FF87
:1010C00004E001228021024805F07EFF10BD0000EF
:1010D0000014014010B5044604F4002030B1002291
:1010E0004FF48061044805F06FFF04E00122910293
:1010F000014805F069FF10BD0014014010B5044619
:1011000004F4802030B100224FF48051044805F0EF
:101110005BFF04E001221103014805F055FF10BDFB
:101120000010014010B5044604F4805028B100229C
:101130000121054805F048FF04E00122114602485C
:1011400005F042FF10BD00000018014010B5044634
:1011500004F0806028B100220421054805F034FF26
:1011600004E001220421024805F02EFF10BD00001A
:101170000010014010B5044604F0100028B1002210
:101180008021054805F020FF04E00122802102486B
:1011900005F01AFF10BD00000010014010B5044614
:1011A00004F0080028B101229103054805F00CFF66
:1011B00005E000224FF48041014805F005FF10BD15
:1011C000001401402DE9F84F05460C462846A16958
:1011D000FFF753F806464E49FFF7CEF903D26420D5
:1011E00084F82D0064E04FF08141A068FFF77AF8A1
:1011F00080464FF081406168FFF774F881464FF0F8
:101200007E51FEF7E5FF07464146FEF7E1FF064641
:101210002168FFF735F8E0614FF08040A168FFF7E3
:101220002FF880464FF08141FFF75CF807464FF0FA
:101230007E51FEF7CDFF06462168FFF721F82062B8
:10124000A1682068FFF71CF806464FF08141FFF7C0
:1012500049F860626069E060206960612846A169C0
:10126000FFF70BF82061E168606AFFF709F800906A
:101270006169206AFFF704F881462169E069FEF799
:10128000FFFF824694F92C00FFF7D9F883465146B8
:10129000FEF79EFF80464946FEF7ECFF07460099A1
:1012A000FEF796FF0646FFF7E9F840B284F82D00F6
:1012B00094F92D00002803DA002084F82D000DE0B9
:1012C00094F92D0094F82E10884202DD94F82E0037
:1012D00001E094F92D0040B284F82D0094F830001C
:1012E000FFF7B6F80746A169FEF772FF06462946E2
:1012F000FFF738F902D2002084F82D002C346078F2
:10130000207094F901002C3C80B2BDE8F88F0000F9
:10131000000048422DE9F04F85B005460C461646C0
:101320006069E060206960612846A169FEF7A5FF59
:1013300020612846A169FEF7A0FF82464849FFF7D1
:101340001BF908D847492846FFF70CF903D250206B
:1013500084F82D005BE04FF08141A068FEF7C2FFEA
:1013600004904FF081406168FEF7BCFF4FF07E5162
:101370000390FEF72DFF83460499FEF729FF82466E
:101380002168FEF77DFF07464FF08040A168FEF719
:1013900077FF4FF081410490FEF7A4FF83464FF0A2
:1013A0007E51FEF715FF82462168FEF769FF8046F1
:1013B000A1682068FEF764FF82464FF08141FEF786
:1013C00091FF81464846E168FEF75AFF0490404687
:1013D0006169FEF755FF039038462169FEF750FF1B
:1013E000019094F92C00FFF72AF800900199FEF77C
:1013F000EFFE02900399FEF73DFF83460499FEF746
:10140000E7FE8246FFF73AF840B284F82D0094F9DF
:101410002D00002803DA002084F82D000AE094F95A
:101420002D00B04201DD304601E094F92D0040B2BC
:1014300084F82D000C49A069FEF7CAFE82462946B1
:10144000FFF790F802D2002084F82D002C34607849
:10145000207094F901002C3C80B205B0BDE8F08FFB
:101460000000484200803B440000A04010B5044604
:10147000A07A3B2817DD0020A072607A401C6072C1
:10148000607A3B280FDD00206072207A401C2072B9
:10149000207A172807DD00202072E078401CE070D9
:1014A000204600F001F810BD1FB5044610A30FCB75
:1014B0008DE80F00E078A1781DF80110884216DD54
:1014C000208807F087FC28B1A078022802D1E078B4
:1014D0001D280CDD0120E070A078401CA070A078D1
:1014E0000C2804DD0120A0702088401C20801FBD36
:1014F0001F1F1C1F1E1F1E1F1F1E1F1E1F00000060
:1015000010B502460B460020114604E00C68641C2E
:1015100004B10846091D9942F8D310BD2DE9F041E8
:101520000026B0460027002422E0601C142190FB16
:10153000F1F201FB1208214800681C3030F8140059
:10154000B0F5805F00DB761C1C4A12681C3232F852
:1015500018101A4A12681C3232F8140001F0FAFE10
:101560000546C82D01DBD22D00DD761C2F44641CFE
:10157000142CDADB40F6FA70874208DA1048808DC6
:1015800040F040000E4988850120BDE8F0810C48FC
:10159000808D20F040000A49888536B10846808D4C
:1015A00040F0400088850120EFE70548808D20F05D
:1015B0004000034988850020E7E700000CCA0008C6
:1015C0006A0F00200448B0F840004CF20C11884328
:1015D0000149A1F8400070476A0F00200448B0F8A4
:1015E00040004CF2301188430149A1F84000704797
:1015F0006A0F002038B53348807AAA2855D131487F
:10160000C07A552851D12F48007B841D2D488088F1
:10161000A0424AD12B4881880A30FFF7FEFB80B1F7
:101620002848828800F10A012748FEF7ADFD2548C9
:101630008088401C40102449091F48800120087000
:1016400033E055201F4981F89A01AA211D4880F8EE
:101650009B11042180F89C11002180F89D1180F8D5
:101660009E1180F89F11102180F8A011802180F830
:10167000A111082100F5CD7009F042F900909DF804
:101680000010104880F8A2119DF8011080F8A311F5
:101690000A200C49C8800846C28800F5CD710B4865
:1016A00007F094F8012005F003FA322105480A30CA
:1016B000FEF783FD322203490A31044807F022F87D
:1016C000002038BDF8010020480A0020AC060020A8
:1016D00030B585B014216846FEF76FFD002407E0A1
:1016E000AF48005D00F07F000DF80400601CC4B23C
:1016F000142CF5DBAA480A388088401E1DF800002B
:101700000A2853D1A6480A388088801E1DF8000098
:101710000D28F6D1A348B0F8400040F48070A149EC
:10172000A1F840000846408D48F2260188439D49B3
:1017300048850846808D20F40050888598480A38EE
:101740008088072877DA9DF80000532838D10846AA
:10175000B0F8400020F40040A1F840009DF80200DD
:101760002D280BD10846B0F8400040F00200A1F847
:1017700040008D488D498968086007E08948B0F8C5
:10178000400020F002008749A1F840009DF80200C7
:101790002B280CD18348B0F8400040F0010081496B
:1017A000A1F840008248814989680860ECE07D48E2
:1017B000B0F8400020F001007A49A1F84000E3E0D1
:1017C0009DF800005A2837D17648B0F8400020F440
:1017D00000407449A1F840009DF80300532812D13D
:1017E0000846B0F8400040F02000A1F8400008464C
:1017F000B0F8400020F01000A1F8400000206B4934
:1018000089680860C0E09DF803004428CED165488F
:10181000B0F8400020F020006249A1F840000846DE
:10182000B0F8400040F01000A1F8400061485F4966
:1018300089680860A8E010E09DF800004528B5D14F
:101840009DF801005328B1D15648B0F8400040F44B
:1018500000405449A1F8400096E05248B0F84000DA
:1018600020F008004F49A1F840000846B0F84000B9
:1018700020F40040A1F840009DF8000053287BD1DF
:101880009DF810000D2877D101204849487045483F
:10189000B0F8400020F003004249A1F840009DF854
:1018A000020053280ED10846B0F8400040F008006E
:1018B000A1F840000846B0F8400020F00400A1F86C
:1018C00040000EE03748B0F8400040F004003549D1
:1018D000A1F840000846B0F8400020F00800A1F848
:1018E000400000203149896808608DF80100052416
:1018F0002AE01DF8040030281DDB1DF804003928FB
:1019000019DC2A49896808682B49FEF7B9FC274980
:10191000896808601DF80410A1F13000FEF78FFD02
:1019200005462248806801682846FEF751FC1F4999
:101930008968086006E01DF804002D2802D1012006
:101940008DF80100601CC4B20E2CD2DB9DF80100A2
:1019500038B116488068006880F0004013498968F3
:1019600008601249896808681449FEF7BBFC0F49F2
:101970008968086008E0FFE70A48B0F8400040F4D2
:1019800080400849A1F8400014210548FEF715FCE5
:1019900003480A3800F01CF8002005B030BD0000F4
:1019A0009A0500206A0F00200000FAC30C0A0020EC
:1019B0000000FA4317B7D1380000204100401C4610
:1019C0000021017081800172C18041728170704775
:1019D0000021017081800172704700002DE9FC41F7
:1019E000054600264FF4C871FE48FEF7E6FBFD4CA5
:1019F000241D27462A894CF60250111A824201F012
:101A0000998073DC4CF60300A2EB000182426ED099
:101A10003CDC4CF24011A2EB01008A4268D01ADC97
:101A20004CF20111A2EB01008A426FD00CDC6FF482
:101A30004040104400286AD0012869D0022868D0AC
:101A4000032841F05B8494E201287DD002287CD0F9
:101A50000328F6D10CE340F2C222811A904275D0DD
:101A60000BDCA0F2C110002871D03E2870D03F28B6
:101A70006FD0B0F5807FE4D1DCE33E296AD0A1F2DB
:101A8000FF31002967D00129DBD1FCE340F2FF12CE
:101A9000881A914201F0E18016DC062901F02683C4
:101AA00008DC012974D0022973D0032972D00529DA
:101AB000C7D1E9E3072901F03B833D296BD0B1F59C
:101AC000FF7FBED101F0A7B8B0F5817F01F04D8155
:101AD0000FDCFF2801F0E380B0F5807F01F0018189
:101AE000A0F201100028ACD101F01DB912E0EEE324
:101AF00099E2A0F20310002801F05981012801F0B9
:101B00007881B0F5FE7F9CD101F002B841E2E1E0BE
:101B100012E11EE240F2FF62881A91427ED045DC5B
:101B200040F23E22A1EB0200914278D01FDCFF2957
:101B300001F0308010DC012972D0022971D0032914
:101B400070D03E2985D1EEE33AE278E221E359E113
:101B50009CE076E0EEE2A6E3B1F5807F01F038800C
:101B6000A1F2FF1100297DD0012984D1F3E3C5281A
:101B700001F0788210DCC12801F00E82C22801F049
:101B8000E981C32801F02A82C42891D101F048BA22
:101B9000F6E3F6E3F6E3F6E3C62801F08582D02803
:101BA00072D0B0F5807F8CD100F062BFB0F5E06FED
:101BB0006BD020DCB0F5007F00F086870FDCB0F53D
:101BC000807F01F03881A0F20110002801F05C81D3
:101BD000012801F07B81022885D101F099B9A0F29A
:101BE0000120002800F08287A0F2FF30002870D08A
:101BF000012888D17EE2B0F5245F01F0FD8212DC7D
:101C0000A0F2017000287DD0A0F50050FF38002818
:101C100001F03683012895D101F051BBF1E0FDE3DD
:101C2000FDE3FDE3FDE36FF424510844002801F0D7
:101C3000FF82FF2801F09E82B0F5807F95D101F0F0
:101C4000BABA4CF2403024F8020B4FF6FF7024F879
:101C5000020B002024F8020B634964480068FEF779
:101C60008BFC00E0FDE307D26148006820F00F0024
:101C7000401C5F49086005E05D48006820F00F00E7
:101C80005B49086001F044BBECE384E04CF23F3078
:101C900024F8020B687868B95548007800F00F0006
:101CA000022807D1002024F8020B48F2010024F892
:101CB000020B0DE04FF6FF7024F8020B002024F811
:101CC000020B4B48006820F00F00C01C4849086018
:101CD000D8E7D9E14CF2010024F8020B4FF6FF706F
:101CE00024F8020B002024F8020B4248008824F854
:101CF000020B4048408824F8020B3E48808824F8B4
:101D0000020B00E05EE03B48C08824F8020B394833
:101D1000008924F8020B3748408924F8020B43F26B
:101D2000316024F8020B44F6352024F8020B4FF6FC
:101D3000FF7024F8020BA5E74CF2020024F8020B16
:101D40004FF6FF7024F8020B002024F8020B2948FC
:101D5000008824F8020B2748408824F8020B254805
:101D6000808824F8020B2348C08824F8020B2148FD
:101D7000008924F8020B1F48408924F8020B43F223
:101D8000316024F8020B44F6352024F8020B0020C1
:101D900024F8020B76E74DF6013024F8020B4FF6DB
:101DA000FF7024F8020B002024F8020B1249D5F82A
:101DB0000A200A60D5F80E0048600846416806F01F
:101DC00093FF5FE74DF6023024F8020B4FF6FF70E9
:101DD00024F8020B002024F8020B07480168216058
:101DE00040680BE092030020000034422C000020E9
:101DF000480000205C0F0020D409002060600834F7
:101E000040E700BF05F10A0001F090FA00287CD0FD
:101E1000F648806C401CF54988644CF2013024F887
:101E2000020B4FF6FF7024F8020B002024F8020B7F
:101E3000EF48C08824F8020BED48408924F8020BD3
:101E4000EB48808924F8020BE948C08924F8020B8A
:101E5000E848C08824F8020BE648408924F8020BC1
:101E6000E448808924F8020BE248C08924F8020B78
:101E7000E148008824F8020BDF480068000C24F8D1
:101E8000020BDE48008824F8020BDC480068000CD6
:101E900024F8020BDA4800680190BDF8040024F829
:101EA000020BBDF8060024F8020BD648006801902A
:101EB000BDF8040024F8020BBDF8060024F8020B5C
:101EC000D148B0F84A0024F8020BCF48B0F84C00D3
:101ED00024F8020BCD4800680190BDF8040024F8F6
:101EE000020BBDF8060024F8020BC94800680190F7
:101EF000BDF8040024F8020BBDF8060024F8020B1C
:101F0000C448007800F00F0000E021E08DF80000E8
:101F1000C148C078401CC0B28DF80100BDF8000077
:101F200024F8020BB848808F24F8020BBB4988695B
:101F3000FEF7BDFA24F8020BB348C08A24F8020B5E
:101F4000B148408D24F8020BAF48808D24F8020B75
:101F500098E64CF2030024F8020B4FF6FF7024F8C9
:101F6000020B002024F8020B40F2031024F8020BAD
:101F700088E64CF2040024F8020B4FF6FF7024F8B8
:101F8000020B002024F8020B4FF4827024F8020B9D
:101F900078E64CF2011024F8020B4FF6FF7024F89B
:101FA000020B002024F8020B002606E09C4830F8C3
:101FB000160024F8020B701C86B2222EF6DB61E6B6
:101FC0004CF2021024F8020B0E2205F10A0194488B
:101FD000FEF711FFF8B1002608E0F01C291D31F8CA
:101FE00010008F4921F81600701C86B20E2EF4DB0B
:101FF0000AF096F8064636B124F8026B4FF6FF70E9
:1020000024F8020B0EE04FF6FF7024F8020B0020BC
:1020100024F8020B06E04FF6FF7024F8020B0020B4
:1020200024F8020B2EE64CF2401024F8020B4FF677
:10203000FF7024F8020B002024F8020B22E64CF279
:10204000031024F8020B4FF6FF7024F8020B002057
:1020500024F8020B002608E006F12200704931F84E
:10206000100024F8020B701C86B2142EF4DB09E673
:102070004CF2041024F8020B4FF6FF7024F8020B08
:10208000002024F8020BFDE54DF6012024F8020B98
:10209000687868B95F48007800F00F00022807D11F
:1020A000002024F8020B48F2010024F8020B20E083
:1020B000002211464DF60120FEF75CFB90B1554819
:1020C0000068000C40F004015248006861F31240BF
:1020D000504908604FF6FF7024F8020B002024F8E6
:1020E000020B06E0002024F8020B48F2020024F85C
:1020F000020BC7E54DF6022024F8020B687868B998
:102100004448007800F00F00022807D1002024F88E
:10211000020B48F2010024F8020B0AE04DF6012000
:1021200008F064FF4FF6FF7024F8020B002024F83B
:10213000020BA7E54CF2404024F8020B687868B91E
:102140003448007800F00F00022807D1002024F85E
:10215000020B48F2010024F8020B19E04CF2024095
:1021600008F044FF4CF2014008F040FF4FF6FF70CA
:1021700024F8020B002024F8020B264800780009FE
:1021800020F004012348006861F30610214908602B
:1021900078E54CF2024024F8020B1E48007800F06B
:1021A0000F00022807D1002024F8020B48F201009A
:1021B00024F8020B3DE0002211464CF20240FEF7EB
:1021C000D9FA90B113480078000940F00401114891
:1021D000006861F306100F4908604FF6FF7024F89D
:1021E000020B002024F8020B23E01BE0EC0E002081
:1021F0006C0D00202C0E00200400002008000020A0
:1022000034000020380000206A0F00202C0000203D
:102210003000002048000020F80000202C010020A1
:10222000CE0F0020002024F8020B48F2020024F810
:10223000020B27E54CF2014024F8020B687868B9DC
:10224000FB48007800F00F00022807D1002024F896
:10225000020B48F2010024F8020B23E00022114691
:102260004CF20140FEF786FAA8B1F1480078000967
:1022700040F00401EE48006861F30610EC49086084
:102280004FF6FF7001E03AE04CE124F8020B002029
:1022900024F8020B06E0002024F8020B48F20200AA
:1022A00024F8020BEEE44CF6010024F8020B6878E7
:1022B00070B9DF48007800F00F00022808D1002034
:1022C00024F8020B48F2010024F8020B16E043E068
:1022D000002211464CF60100FEF74CFA38B14FF6D9
:1022E000FF7024F8020B002024F8020B06E0002007
:1022F00024F8020B48F2020024F8020BC2E44CF668
:10230000020024F8020B687870B9C948007800F020
:102310000F00022808D1002024F8020B48F2010027
:1023200024F8020B16E09CE2002211464CF6020053
:10233000FEF720FA38B14FF6FF7024F8020B0020A8
:1023400024F8020B06E0002024F8020B48F20200F9
:1023500024F8020B96E48FE14CF6030024F8020BFC
:10236000687888B9B248007800F00F0002280BD1D5
:10237000002024F8020B48F2010024F8020B24E0AC
:1023800024E05EE098E003E1002211464CF60300F1
:10239000FEF7F0F990B14FF6FF7024F8020B002021
:1023A00024F8020BA2480068000C40F00401A04889
:1023B000006861F312409E49086006E0002024F89E
:1023C000020B48F2020024F8020B5BE44CF6040016
:1023D00024F8020B687868B99548007800F00F007F
:1023E000022807D1002024F8020B48F2010024F84B
:1023F000020B25E0002211464CF60400FEF7BAF964
:10240000B8B14FF6FF7024F8020B002024F8020B3D
:1024100087480068000C40F0040103E062E190E1AD
:10242000BFE1EEE18248006861F312408049086034
:1024300006E0002024F8020B48F2020024F8020B08
:1024400020E44CF6050024F8020B687880B978483F
:10245000007800F00F0002280AD1002024F8020BB7
:1024600001E0D0E038E248F2010024F8020B22E05B
:102470006889401E81B200224CF60500FEF77AF909
:1024800090B14FF6FF7024F8020B002024F8020BE5
:1024900067480068000C40F004016548006861F37B
:1024A00012406349086006E0002024F8020B48F25D
:1024B000020024F8020B0BE44CF6060024F8020B91
:1024C000687868B95A48007800F00F00022807D1F0
:1024D000002024F8020B48F2010024F8020B20E04F
:1024E000002211464CF60600FEF744F990B14FF673
:1024F000FF7024F8020B002024F8020B4C480068FF
:10250000000C40F004014A48006861F31240484959
:10251000086006E0002024F8020B48F2020024F8CC
:10252000020B08E44CF6080024F8020B687868B93E
:102530003F48007800F00F00022807D1002024F85F
:10254000020B48F2010024F8020B20E000221146A1
:102550004CF60800FEF70EF990B14FF6FF7024F824
:10256000020B002024F8020B31480068000C40F0F8
:1025700004012F48006861F312402D49086006E00D
:10258000002024F8020B48F2020024F8020B18E4A1
:102590004CF6400024F8020B687868B924480078AB
:1025A00000F00F00022807D1002024F8020B48F2A7
:1025B000010024F8020B25E04CF6030008F016FD9C
:1025C0004CF6040008F012FD4CF6050008F00EFD74
:1025D0004CF6080008F00AFD4CF6060008F006FD6F
:1025E00013480068000C20F004011148006861F3F2
:1025F00012400F4908604FF6FF7024F8020B0020CC
:1026000024F8020BA4E44CF6017024F8020B68785D
:1026100080B90748007800F00F0002280AD1002096
:1026200024F8020B48F2010024F8020B23E000001A
:1026300048000020002211464CF60170FEF79AF87F
:1026400090B14FF6FF7024F8020B002024F8020B23
:10265000F9480088400B40F00401F748006861F336
:102660004F30F549086006E0002024F8020B48F2DC
:10267000020024F8020B6BE44CF6027024F8020B03
:10268000687868B9EC48007800F00F00022807D19C
:10269000002024F8020B48F2010024F8020B20E08D
:1026A000002211464CF60270FEF764F890B14FF626
:1026B000FF7024F8020B002024F8020BDE4800888B
:1026C000400B40F00401DC48006861F34F30DA4908
:1026D000086006E0002024F8020B48F2020024F80B
:1026E000020B35E44CF6407024F8020B687868B9A8
:1026F000D148007800F00F00022807D1002024F80C
:10270000020B48F2010024F8020B19E04CF60270AB
:1027100008F06CFC4CF6017008F068FCC6480088B4
:10272000400B20F00401C448006861F34F30C249F7
:1027300008604FF6FF7024F8020B002024F8020B0B
:1027400006E44CF6035024F8020B687868B9BA48DE
:10275000007800F00F00022807D1002024F8020BB7
:1027600048F2010024F8020B1AE04CF60350B3497A
:10277000C8800020C8818881022008624FF6FF705F
:1027800024F8020B002024F8020BAB480068C00CB0
:1027900040F00401A848006861F3D540A6490860EC
:1027A0000DE44CF6045024F8020B687868B9A2488E
:1027B000007800F00F00022807D1002024F8020B57
:1027C00048F2010024F8020B1AE04CF604509B4931
:1027D000C8800020C8818881032008624FF6FF70FE
:1027E00024F8020B002024F8020B93480068C00C68
:1027F00040F004019048006861F3D5408E490860BC
:1028000010E44CF6055024F8020B687868B98A4841
:10281000007800F00F00022807D1002024F8020BF6
:1028200048F2010024F8020B1AE04CF605508349E7
:10283000C8800020C8818881012008624FF6FF709F
:1028400024F8020B002024F8020B7B480068C00C1F
:1028500040F004017848006861F3D540764908608B
:1028600005E44CF6405024F8020B687868B97248C9
:10287000007800F00F00022807D1002024F8020B96
:1028800048F2010024F8020B25E04CF640506B4959
:10289000C8804FF6F070488167480068C00C20F08F
:1028A00004016548006861F3D540634908606448E5
:1028B000006820F080406249086000206149C968D2
:1028C00008606049496808604FF6FF7024F8020B01
:1028D000002024F8020B0CE44DF2100024F8020B47
:1028E000687868B95448007800F00F00022807D1D2
:1028F000002024F8020B48F2010024F8020B99E0B2
:102900006889FDF7A5FD5049886188694F49FDF741
:1029100029FE17D24C4988690021FDF72DFE11D2FE
:102920004B48494908604B4848604B488860084616
:10293000416B88471E20444981F82E00012081F810
:102940002F0070E0404988694449FDF70BFE18D21A
:102950003D4988693D49FDF70FFE12D84FF082408E
:10296000394908603E484860400288600846416B2B
:1029700088475020344981F82E00012081F82F002B
:1029800051E0314988693749FDF7ECFD18D22E49ED
:1029900088693249FDF7F0FD12D84FF082402A498C
:1029A00008602F484860400288600846416B8847AD
:1029B0005A20254981F82E00012081F82F0032E0AD
:1029C000214988692749FDF7D7FD05D91E4988693E
:1029D0002549FDF7C7FD17D200201B49886181F802
:1029E0002F002248006820F0007020490860084647
:1029F000006820F080600860002024F8020B48F294
:102A0000BA0024F8020B14E400200F4981F82F00CB
:102A10001648006820F000701449086008460068F5
:102A200020F0806008604FF6FF7024F8020B002051
:102A300024F8020B36E40000480000202C0E002091
:102A4000040000200C0A00202C0100200000484354
:102A500000007041000016430000A0410000164431
:102A60000000204200008C44000020C1080000202B
:102A70004DF2400024F8020B687868B9F8480078F5
:102A800000F00F00022807D1002024F8020B48F2C2
:102A9000010024F8020B16E00020F249886181F859
:102AA0002F00F148006820F00070EF4908600846E8
:102AB000006820F0806008604FF6FF7024F8020B79
:102AC000002024F8020B19E44DF2016024F8020BF7
:102AD000E548006840F40060E34908604FF6FF7085
:102AE00024F8020B002024F8020B07E44DF20260E8
:102AF00024F8020BDC48006820F40060DA49086022
:102B00004FF6FF7024F8020B002024F8020BFFE3BD
:102B10004CF6015024F8020B4FF6FF7024F8020B1C
:102B2000002024F8020BD048006840F48000CE4911
:102B30000860EDE34CF6025024F8020B687868B99F
:102B4000C748007800F00F00022807D1002024F8C1
:102B5000020B48F2010024F8020B1AE0C04800689A
:102B6000C00C00F0040038B1002024F8020B48F239
:102B7000020024F8020B0CE0BB48006820F480003F
:102B8000B94908604FF6FF7024F8020B002024F8C2
:102B9000020BBDE34CF6016024F8020B687868B9BB
:102BA000AF48007800F00F00022807D1002024F879
:102BB000020B48F2010024F8020B08E008F09AF931
:102BC0004FF6FF7024F8020B002024F8020B9FE35D
:102BD0004CF6026024F8020B687868B9A0480078C7
:102BE00000F00F00022807D1002024F8020B48F261
:102BF000010024F8020B0DE000231A4603214CF6D5
:102C00000260FDF7E1FD4FF6FF7024F8020B002093
:102C100024F8020B7CE34CF6012024F8020B6878C0
:102C200068B98F48007800F00F00022807D1002013
:102C300024F8020B48F2010024F8020B0CE08A4849
:102C4000006840F40050884908604FF6FF7024F88F
:102C5000020B002024F8020B5AE34CF6022024F861
:102C6000020B687868B97E48007800F00F000228EF
:102C700007D1002024F8020B48F2010024F8020BCF
:102C80000CE07948006820F40050774908604FF65E
:102C9000FF7024F8020B002024F8020B38E34CF6F6
:102CA000013024F8020B687868B96D48007800F0AC
:102CB0000F00022807D1002024F8020B48F201007F
:102CC00024F8020B0CE06848006840F40070664984
:102CD00008604FF6FF7024F8020B002024F8020B66
:102CE00016E34CF6023024F8020B687868B95C48A9
:102CF000007800F00F00022807D1002024F8020B12
:102D000048F2010024F8020B0CE05748006820F458
:102D10000070554908604FF6FF7024F8020B002040
:102D200024F8020BF4E24CF6033024F8020B687826
:102D300068B94B48007800F00F00022807D1002046
:102D400024F8020B48F2010024F8020B0CE046487C
:102D5000006840F48060444908604FF6FF7024F832
:102D6000020B002024F8020BD2E24CF6043024F8C7
:102D7000020B687868B93A48007800F00F00022822
:102D800007D1002024F8020B48F2010024F8020BBE
:102D90000CE03548006820F48060334908604FF645
:102DA000FF7024F8020B002024F8020BB0E24CF66E
:102DB000053024F8020B687868B92948007800F0DB
:102DC0000F00022807D1002024F8020B48F201006E
:102DD00024F8020B0CE02448006840F4807022497B
:102DE00008604FF6FF7024F8020B002024F8020B55
:102DF0008EE24CF6063024F8020B687868B9184861
:102E0000007800F00F00022807D1002024F8020B00
:102E100048F2010024F8020B0CE01348006820F48B
:102E20008070114908604FF6FF7024F8020B0020F3
:102E300024F8020B6CE24DF2015024F8020B687882
:102E4000A0B90748007800F00F0002280ED100203A
:102E500024F8020B48F2010024F8020B13E00000F2
:102E6000480000202C01002008000020FA480068DB
:102E700040F48050F84908604FF6FF7024F8020BC8
:102E8000002024F8020B43E24DF2025024F8020B1A
:102E9000687868B9F148007800F00F00022807D17F
:102EA000002024F8020B48F2010024F8020B0CE089
:102EB000E948006820F48050E74908604FF6FF7049
:102EC00024F8020B002024F8020B21E24DF20350FB
:102ED00024F8020B687868B9E048007800F00F0029
:102EE000022807D1002024F8020B48F2010024F840
:102EF000020B0CE0D848006840F40000D649086096
:102F00004FF6FF7024F8020B002024F8020BFFE1BB
:102F10004DF2045024F8020B687868B9CF48007865
:102F200000F00F00022807D1002024F8020B48F21D
:102F3000010024F8020B0CE0C748006820F40000F0
:102F4000C54908604FF6FF7024F8020B002024F8F2
:102F5000020BDDE14DF2020024F8020B687868B93B
:102F6000BE48007800F00F00022807D1002024F8A6
:102F7000020B48F2010024F8020B0CE0B64800688E
:102F800020F00070B44908604FF6FF7024F8020B7F
:102F9000002024F8020BBBE14DF2010024F8020BE3
:102FA000687868B9AD48007800F00F00022807D1B2
:102FB000002024F8020B48F2010024F8020B0CE078
:102FC000A548006840F00070A34908604FF6FF7004
:102FD00024F8020B002024F8020B99E14DF20300C3
:102FE00024F8020B687868B99C48007800F00F005C
:102FF000022807D1002024F8020B48F2010024F82F
:10300000020B0CE09448006840F080609249086030
:103010004FF6FF7024F8020B002024F8020B77E132
:103020004DF2040024F8020B687868B98B480078E8
:1030300000F00F00022807D1002024F8020B48F20C
:10304000010024F8020B0CE08348006820F0806047
:10305000814908604FF6FF7024F8020B002024F825
:10306000020B55E14DF2050024F8020B687868B9AF
:103070007A48007800F00F00022807D1002024F8D9
:10308000020B48F2010024F8020B0CE072480068C1
:1030900040F08070704908604FF6FF7024F8020B12
:1030A000002024F8020B33E14DF2060024F8020B55
:1030B000687868B96948007800F00F00022807D1E5
:1030C000002024F8020B48F2010024F8020B0CE067
:1030D0006148006820F080705F4908604FF6FF701B
:1030E00024F8020B002024F8020B11E14CF6090031
:1030F00024F8020B687868B95848007800F00F008F
:10310000022807D1002024F8020B48F2010024F81D
:10311000020B0CE05048006840F010004E49086077
:103120004FF6FF7024F8020B002024F8020BEFE0AA
:103130004CF60A0024F8020B687868B94748007812
:1031400000F00F00022807D1002024F8020B48F2FB
:10315000010024F8020B0CE03F48006820F010004A
:103160003D4908604FF6FF7024F8020B002024F858
:10317000020BCDE04FF6016024F8020B687868B9C5
:103180003648007800F00F00022807D1002024F80C
:10319000020B48F2010024F8020B0BE00120304939
:1031A0000870FDF7C5FB4FF6FF7024F8020B0020F6
:1031B00024F8020BACE04FF6026024F8020B6878AA
:1031C00068B92648007800F00F00022807D10020D7
:1031D00024F8020B48F2010024F8020B0BE0002057
:1031E0001F490870FDF7A4FB4FF6FF7024F8020B8F
:1031F000002024F8020B8BE04FF6015024F8020B5C
:10320000687868B91548007800F00F00022807D1E7
:10321000002024F8020B48F2010024F8020B06E01B
:103220004FF6FF7024F8020B002024F8020B6FE029
:103230004FF6025024F8020B687898B907480078D6
:1032400000F00F0002280DD1002024F8020B48F2F4
:10325000010024F8020B12E00800002048000020C2
:10326000BC0900202E48006820F000402C4908606E
:103270004FF6FF7024F8020B002024F8020B47E001
:103280004FF6014024F8020B687868B925480078A9
:1032900000F00F00022807D1002024F8020B48F2AA
:1032A000010024F8020B09E068891F4908804FF6E5
:1032B000FF7024F8020B002024F8020B28E04FF6E0
:1032C000024024F8020B687868B91648007800F0CC
:1032D0000F00022807D1002024F8020B48F2010059
:1032E00024F8020B09E000200F4908804FF6FF7018
:1032F00024F8020B002024F8020B09E0002024F837
:10330000020B24F8020B48F2110024F8020B00BF54
:1033100000BFE11BC1F34F0007F06CF8BDE8FC8172
:1033200004000020480000201E000020024600216A
:103330000AE0074830F8110032F81130984201D005
:1033400000207047481CC1B20629F2DB0120F8E7D3
:103350005C0F002002468A4201DD531A00E08B1AFE
:1033600098B2B0F5006F02DDC0F5805398B2704797
:1033700070B504460D4629462046FDF7FDF804D2F7
:1033800029462046FCF776FF03E029462046FCF755
:1033900074FF0646FDF78BF880B270BD02468A4284
:1033A00001DD501A00E0881A80B2704710B502485B
:1033B00003F01AF910BD00000409002010B50248FE
:1033C00003F012F910BD00004809002010B50248B2
:1033D00003F00AF910BD00003808002010B50248BB
:1033E00003F002F910BD0000F407002010B50248F8
:1033F00003F0FAF810BD00007C08002010B5024868
:1034000003F0F2F810BD0000C008002010B502481B
:1034100003F0EAF810BD00006C07002010B5024868
:1034200003F0E2F810BD0000B007002030B590F8BE
:1034300040500124AC40C56B6C6004686360446814
:10344000102C04D10468A2600468E16003E0046801
:10345000A1600468E26030BD7047000010B504460A
:103460006089142832D004DC01280AD00A2854D1FB
:103470000EE01E2844D0A0F57F40F03800284CD143
:1034800047E0002060710A206081002060614AE00E
:10349000002060712548008800F4004038B1002207
:1034A00011464CF60270FDF723FA607106E0002227
:1034B00011464CF60170FDF71BFA6071607900B996
:1034C00031E014206081002060612CE061791848AF
:1034D00050F8210040894FF6FF7188420FD1617981
:1034E000134850F82100C08928B148F20C01204649
:1034F000E26B904703E0002060611E20608112E0D3
:103500006069401C60616069282801D90A206081D7
:1035100009E02046A16B884705E048F204012046F7
:10352000E26B904700BF00BF10BD00000400002008
:10353000400F002000BF011EA0F10100FBD1704729
:10354000C10000BF0A1EA1F10101FBD170470000BC
:103550007FB506460D469F48FEF732FA082E0ED27A
:10356000DFE806F00D040E6A9FA6C5E01F229A4907
:1035700098483C30FCF708FEE8B200F0CFFAFFE0D4
:103580001F22964993483C30FCF7FEFD944890F882
:10359000400000F0010048B148218E4880F84A10F0
:1035A000002180F8561080F85A1044E08C4890F8BA
:1035B000400000F0020048B14C21864880F84A10D3
:1035C000002180F8561080F85A1034E0002D09DAF6
:1035D000804890F8560040F002017E4880F856106E
:1035E0006D4207E07B4890F8560040F001017948B1
:1035F00080F856102A467BA101A808F0A5F80024FF
:1036000005E000222046611CCCB201A90A5401A8A1
:10361000005D302801D1022CF3DB002409E001A871
:10362000015D0A2000EB44026A483C308154601C72
:10363000C4B2072CF3DBA3E01F226C4965483C3081
:10364000FCF7A2FD002D09DA624890F8560040F020
:103650000201604880F856106D4207E05D4890F81E
:10366000560040F001015B4880F856102A4660A1E0
:1036700001A808F069F89DF80410564880F84A102F
:103680009DF8051080F84C109DF8061080F84E103B
:103690009DF8071080F850109DF8081080F852101F
:1036A0006EE01F2253494B483C30FCF76DFD67E04C
:1036B0001F22494947483C30FCF766FD4848808E48
:1036C00000904748438E028E4BA101A808F03CF8B9
:1036D000002409E001A8015D082000EB44023D48F8
:1036E0003C308154601CC4B2082CF3DB48E01F223C
:1036F000394938483C30FCF747FD3948828D41A1B3
:1037000001A808F021F8002409E001A8015D0820C3
:1037100000EB44022F483C308154601CC4B2082C9A
:10372000F3DB2DE01F222C492A483C30FCF72CFD0E
:10373000002D09DA274890F8560040F0020125488C
:1037400080F856106D4207E0224890F8560040F08D
:103750000101204880F856102A462DA101A807F043
:10376000F3FF002409E001A8015D082000EB4402FA
:1037700018483C308154601CC4B2082CF3DB00BFF5
:1037800000BF174890F83E0000F0800038B911489B
:1037900090F8560040F004010E4880F856101F21A2
:1037A0000C483C3007F0ACF8ADF804009DF805106B
:1037B000084880F85B109DF8041080F85C10212008
:1037C0000449C8800846C2883C31124804F0FEFF14
:1037D0007FBD000022050020F2C7000830C80008A5
:1037E0006A0F0020253037640000000011C800086F
:1037F000253564004FC8000825346425303264251F
:1038000030326400455252202530347800000000E8
:1038100025386400EC06002010B5C4880C43C48031
:103820000381202912D006DC042909D0082909D0F7
:10383000102911D108E040290AD080290CD109E0D3
:1038400002740BE0427409E0C26007E0428205E0C6
:10385000828203E0C28201E0C26000BF00BF10BDEF
:1038600070B504460125012609E0E088284000B132
:1038700007E04FF6FF7000EA4505701C86B2102E77
:10388000F3DB00BF208910B12089401E2081102D5C
:1038900036D008DC012D0ED0022D18D0042D63D0B7
:1038A000082D6FD139E0202D1DD0802D4FD0B5F5DA
:1038B000807F67D13EE00120FDF73AF8208928B9E2
:1038C000607818B9E08820F00100E0805BE000201B
:1038D000FDF72EF8208928B9607818B9E08820F023
:1038E0000200E0804FE0618A0320FFF731FE20896B
:1038F00028B9607818B9E08820F02000E08042E024
:103900000220E168FFF724FE208928B9607818B901
:10391000E08820F01000E08035E0617C0120FFF7B6
:1039200017FE208928B9607818B9E08820F00800CF
:10393000E08028E0208928B9607818B9E08820F470
:103940008070E08000210420FFF702FE1BE0208948
:1039500028B9607818B9E08820F08000E080002164
:103960000520FFF7F5FD0EE0208928B9607818B929
:10397000E08820F00400E08000210620FFF7E8FD49
:1039800001E0FFE700BF00BF70BD000038B504468E
:10399000002008490860084684600120C86048602B
:1039A00003F050F96946034803F092F803F0E8F891
:1039B00038BD0000401000200021074AD1610749AE
:1039C000096941F00401054A11611146096941F094
:1039D0004001116170470000A0000020002002405B
:1039E0000021074AD1610749096941F00201054AEE
:1039F000116111464861096941F040011161704748
:103A0000A0000020002002400022054BDA61054A98
:103A1000126942F00102034B1A61018070470000F5
:103A2000A00000200020024000201E49C96801F0CB
:103A3000100139B11C49C96941F002011A4AD1612A
:103A400040F010001749C96801F0040139B1164966
:103A5000C96941F00101144AD16140F004001149E3
:103A6000C96901F0010169B10F49C96941F0040157
:103A70000D4AD16100BF0B49C96921F00101094A12
:103A8000D16100BF00BF40F20111884206D1054953
:103A9000C96921F00101034AD16101E00149C8600F
:103AA00000BF704700200240A000002070B504460F
:103AB00003F090FA054609E0601C38B124B103F028
:103AC00089FA401BA04201D9032070BD1248C0688A
:103AD00000F001000028EFD10F48C06800F020007E
:103AE00020B100BF20200C49C86000BF0A48C06850
:103AF00000F0100048B90848C06900F0010020B982
:103B00000548C06800F0040018B1FFF78DFF0120E0
:103B1000DBE70020D9E700000020024010B50021BB
:103B200008220AE000EBC003084C23445C5C084B0D
:103B30009C54931CDAB24B1CD9B200EBC003034C6B
:103B400023445B5C002BEDD110BD00006EC8000863
:103B50005E0500202DE9F04180460FFA88F42648E2
:103B60000068808B201A04B2002C02DA04F5805021
:103B700004B2D22094FBF0F0C5B200261EE01E492C
:103B800009681C3131F815004146FFF7E3FB07B225
:103B9000681C142190FBF1F201FB1200C5B216491A
:103BA00009681C3131F815004146FFF7D3FB04B218
:103BB0003819DC2800DA03E0701CC6B2022EDEDB06
:103BC00000BF022E14DAA7420BDA05F1130014210C
:103BD00090FBF1F201FB1204072F0ADD44F0800490
:103BE00007E0072C01DA2C4603E045F0800400E0F2
:103BF000FF24E0B2BDE8F0810CCA000810B504460D
:103C00006089012809D0642817D0782825D0A0F52C
:103C10007F40F03800286BD145E06420608149483E
:103C2000006820F40040474908600846006820F416
:103C3000804008600020606181E06069401C606134
:103C4000282809D93F48006840F480403D49086071
:103C5000782060810020606171E06069401C6061D3
:103C6000B0F5397F1ED93748006820F480403549C7
:103C7000086035480088400B20F004013248006895
:103C800061F34F30304908602046A16B88472F48C8
:103C9000006840F480402D4908600846006820F420
:103CA000004008604BE02748006820F400402549A8
:103CB00008600846006820F48040086022480088B8
:103CC000400B20F004012048006861F34F301E498A
:103CD00008601E48006820F480401C4908600846BF
:103CE000006820F4004008602046A16B884726E069
:103CF0001448006820F40040124908600846006833
:103D000020F48040086010480088400B20F0040137
:103D10000D48006861F34F300B4908600B4800689C
:103D200020F48040094908600846006820F40040FB
:103D3000086048F264012046E26B904700BF00BF74
:103D400010BD0000080000204800002004000020F2
:103D500010B504466089012809D0642817D06E2860
:103D600025D0A0F57F40F038002871D14AE04D48B9
:103D7000006840F400404B4908600846006820F4A1
:103D800080400860642060810020606187E0606995
:103D9000401C6061282809D94248006840F48040EE
:103DA000404908606E2060810020606177E06069B2
:103DB000401C6061B0F5207F23D93A48006820F4A8
:103DC0000040384908600846006820F480400860D8
:103DD00035480088400B20F004013348006861F347
:103DE0004F30314908602046A16B88472F48006852
:103DF00040F400402D4908600846006820F48040E7
:103E000008604CE02748006820F40040254908601D
:103E10000846006820F48040086023480088400B72
:103E200020F004012048006861F34F301E4908600B
:103E30001E48006820F400401C49086008460068DD
:103E400020F4804008602046A16B884727E0FFE708
:103E50001448006820F400401249086008460068D1
:103E600020F48040086048F204012046E26B90474D
:103E70000D480088400B20F004010B48006861F3F6
:103E80004F30094908600948006820F4004007499C
:103E900008600846006820F48040086000BF00BF4A
:103EA00010BD000008000020480000200400002091
:103EB00010B504466089B0F5967F73D010DC0A28EF
:103EC00043D006DC012822D002282BD003287DD144
:103ED00032E01E2842D028284BD03228F7D154E0B7
:103EE000B0F5FA7F73D009DCB0F59B7F78D0B0F5E0
:103EF000C87F6ED0B0F5CD7FE9D18AE0B0F5FF7F05
:103F000068D0A0F57F40F0380028E0D1B2E0012071
:103F100007F022F8022007F01FF80220608100203D
:103F20006061B1E06069401C60610A2803D9032028
:103F3000608100206061A7E00021084600F04AFC93
:103F40000A206081002060619EE06069401C606121
:103F50006069282801D91E20608195E04B480078CF
:103F60000A2802DD2820608102E04FF4967060810B
:103F70008AE04748007800F0080018B14FF4C87094
:103F8000608101E0322060817EE0404880790A282B
:103F900004DA4FF4FA70608103E003E02046A16B7D
:103FA000884771E0002211464CF20140FCF7A0FC6A
:103FB0006071607998B14FF49B70608135480078EA
:103FC000000940F004013348006804E056E02CE0AA
:103FD00006E011E041E061F306102E49086053E06D
:103FE00061792D4850F8210040894FF6FF718842D1
:103FF00001D12820608147E0002211464CF60200E2
:10400000FCF776FC6071607910B14FF4CD7060817F
:104010003AE06179204850F8210040894FF6FF715D
:10402000884201D1322060812EE0002211464CF6F8
:104030000270FCF75DFC6071607968B14FF4FF704D
:10404000608114480088400B40F00401114800686A
:1040500061F34F300F49086016E061790E4850F85F
:10406000210040894FF6FF71884202D12046A16BA2
:10407000884709E02046A16B884705E048F2040123
:104080002046E26B904700BF00BF10BD8C090020A6
:104090000C00002048000020400F002010B504460E
:1040A00060898C2879D00EDC5A2877D006DC01286C
:1040B00021D0022873D00A2872D1A2E0642870D0DF
:1040C0006528F9D1DAE0B0F57E4F6BD009DC96288F
:1040D00069D0A02868D06FF4704108440028EBD163
:1040E00079E16FF47E410844002875D0A0F2EF100A
:1040F0000028E1D1B5E1F74840780A280EDDF648FE
:104100000078000920F00401F348006861F306100C
:10411000F14908602046A16B8847D8E1EF4890F844
:104120002C0000F0010080B1EB480078000920F07D
:104130000401E948006861F30610E749086048F2A5
:104140000C012046E26B9047C1E1E44890F82C0056
:1041500000F0400050B1E2484089002806DDE04808
:104160004089032802DC02206081B0E1DB4890F83E
:104170002C0000F04000C0B1D7480078000920F0C2
:104180000401D548006861F30610D349086048F27D
:104190000A012046E26B904799E179E04EE026E083
:1041A00079E15BE049E1B9E0E3E0CB480068000C6D
:1041B00000F0040088B1C8480078000920F004012C
:1041C000C548006861F30610C349086048F246011B
:1041D0002046E26B90477AE139E1BE4840692061B0
:1041E00000206070207160610A2060816FE1B94831
:1041F0004069206100206070207160610A20608148
:1042000065E1B448C0790A2802DD5A2060815EE188
:104210006069401C606128280FD9AF480078000908
:1042200020F00401AC48006861F30610AA49086058
:1042300048F290012046E26B904748E1A9480068A7
:1042400020F40030A74908600846006820F4803058
:104250000860642060810020606138E16069401C72
:104260006061282809D99F48006840F480309D4942
:104270000860652060810020606128E16069401C61
:104280006061282803D98C206081002060611EE1D4
:10429000904840692169401AB0F5966F1BD9914842
:1042A000006820F400308F4908600846006820F458
:1042B0008030086088480078000920F004018648B2
:1042C000006861F306108449086048F277012046CF
:1042D000E26B9047FBE07F48C0790A280EDA8148FC
:1042E000006820F480307F490860002060614FF44E
:1042F0007E4060814FF201002085E8E075484078FB
:1043000004280ADD7748006820F480307549086089
:104310000020606196206081D9E0D8E06D48407847
:104320000A2807DD002060614FF601606081A0204F
:104330002085CCE06069401C6061282818D920796C
:10434000401C20712079052810DD634800780009A1
:1043500020F004016048006861F306105E490860BF
:1043600048F2B7012046E26B9047B0E05A206081E6
:10437000ADE0584840780A280EDD5748007800091B
:1043800020F004015448006861F3061052490860A7
:104390002046A16B88479AE06069401C606128282C
:1043A00018D92079401C20712079052810DD4A4851
:1043B0000078000920F004014748006861F3061006
:1043C0004549086048F2B7012046E26B90477EE01D
:1043D0005A2060817BE06078401CC0B26070142875
:1043E0001BDD4048006820F400303E490860084664
:1043F000006820F48030086037480078000920F019
:1044000004013548006861F306103349086048F23A
:1044100090012046E26B904759E02E48C0790A2867
:1044200008DA002060614FF47E4060814FF20100A5
:10443000208501E05A20608149E06069401C60618C
:10444000282803D900206061208D60813FE06069E9
:10445000401C6061142803D900206061208D6081B8
:1044600035E02048006820F400301E490860084606
:10447000006820F48030086017480078000920F0B8
:1044800004011548006861F30610134908602046CE
:10449000A16B88471BE01348006820F400301149E5
:1044A00008600846006820F4803008600A480078F8
:1044B000000920F004010848006861F3061006496D
:1044C000086048F261012046E26B904700BF00BFE0
:1044D00010BD00008C090020480000206A0F002059
:1044E000F80000200800002010B5044660896E28FE
:1044F00070D008DC012814D05A285BD064286DD015
:10450000652869D17CE0782867D0822876D06FF45E
:104510007E410844002872D0A0F2EF100028F0D1AC
:1045200017E1A84800780A280EDDA748007800099E
:1045300020F00401A448006861F30610A249086055
:104540002046A16B88473AE1A04890F82C0000F083
:10455000010080B19C480078000920F004019A48CD
:10456000006861F306109849086048F20C01204683
:10457000E26B904723E194480068000C00F00400CF
:1045800080B191480078000920F004018E4800684D
:1045900061F306108C49086048F246012046E26B40
:1045A00090470CE1874840692061002020715A2023
:1045B000608104E18648006840F400308449086066
:1045C0000846006820F48030086064206081002084
:1045D0006061F4E01EE001E0D5E053E06069401C5A
:1045E0006061282809D97A48006840F48030784909
:1045F00008606520608100206061E0E06DE09EE081
:104600006069401C6061282803D96E206081002009
:104610006061D4E06B4840692169401AB0F5966F3B
:104620001BD96B48006820F40030694908600846CF
:10463000006820F48030086063480078000920F0AA
:1046400004016148006861F306105F49086048F2A0
:1046500078012046E26B9047B1E05A480078042880
:104660000FDD5B48006820F40030594908600846B7
:10467000006820F48030086000206061782060814C
:104680009DE09CE04F4800780A2807DD002060612B
:104690004FF6016060818220208590E06069401CB7
:1046A0006061282818D92079401C207120790528BC
:1046B00010DD45480078000920F0040142480068F8
:1046C00061F306104049086048F2B8012046E26BE9
:1046D000904774E05A20608171E03A4800780A28D7
:1046E0000EDD39480078000920F0040136480068E2
:1046F00061F30610344908602046A16B88475EE0EC
:104700006069401C6061282818D92079401C2071FC
:104710002079052810DD2C480078000920F00401DC
:104720002948006861F306102749086048F2B8017B
:104730002046E26B904742E05A2060813FE060698A
:10474000401C6061142803D900206061208D6081C5
:1047500035E01F48006820F400301D490860084615
:10476000006820F48030086017480078000920F0C5
:1047700004011548006861F30610134908602046DB
:10478000A16B88471BE01248006820F400301049F4
:1047900008600846006820F4803008600A48007805
:1047A000000920F004010848006861F3061006497A
:1047B000086048F261012046E26B904700BF00BFED
:1047C00010BD00008C090020480000206A0F002066
:1047D0000800002070B504460D46B4B115480068C5
:1047E000000C40F004011348006861F312401149C5
:1047F00008600120104948700846857000208882B2
:1048000000210E4803F062FC12E00A480068000C28
:1048100020F004010748006861F312400549086070
:1048200000200549487088700021044803F074FC9A
:1048300070BD000048000020F8000020B8010020F2
:1048400070B50446618982297DD00CDC5A297BD061
:1048500004DC01291AD00A2977D137E0642975D000
:104860006E29F9D1B1E04FF20102881A91426ED05F
:1048700004DC8C296CD09629EED1FEE0A0F6FF5026
:10488000002866D0B0F5F87FE6D16DE1CB4890F80E
:104890002C0000F0010080B148F20C012046E26BD0
:1048A0009047C7480068000C20F00401C448006825
:1048B00061F31240C24908607EE1C248406920614C
:1048C0000020207160700A20608175E1BE48007888
:1048D00000F0080080B948F291012046E26B904751
:1048E000B7480068000C20F00401B548006861F387
:1048F0001240B34908605FE1B24800780A2810DA34
:10490000AF480068000C20F00401AD48006861F376
:104910001240AB49086048F292012046E26B904792
:104920004AE1A7480078000900F00400C0B1A4489B
:104930000068000C20F00401A148006861F31240F7
:104940009F49086006E04CE00FE020E12EE0D8E04F
:1049500089E0FFE048F243012046E26B90472BE1FB
:10496000002060615A20608126E19648007A0A287A
:1049700006DD9648408995490882642060811BE1E4
:104980006069401C606128280FD98D480068000CC0
:1049900020F004018A48006861F3124088490860E9
:1049A00048F248012046E26B904705E14FF4207041
:1049B000864948828648006840F0100084490860B3
:1049C0006E20608100206061F6E06069401C6061DB
:1049D000142805D900210120FFF7FCFE8220608108
:1049E000EAE0784840692169401AB0F5966F14D919
:1049F00000210846FFF7EEFE71480068000C20F029
:104A000004016F48006861F312406D49086048F284
:104A100070012046E26B9047CEE06A4800780A2891
:104A200014DA00210846FFF7D5FE65480068000C3F
:104A300020F004016248006861F312406049086098
:104A400048F292012046E26B9047B5E05F4840781B
:104A500000B1B1E000210846FFF7BCFE0020A061D4
:104A60008C206081A8E0A069401CA061142803D9B3
:104A70000020A061962060819EE05248007A0A28BA
:104A800029DD524A118A5089FEF764FC05B2C82D0F
:104A900010DDD22D0EDA4A480068000C20F0040127
:104AA0004748006861F31240454908602046A16B01
:104AB000884781E042480068000C20F0040140482B
:104AC000006861F312403E49086048F2B001204698
:104AD000E26B904770E0A069401CA06150280FD99C
:104AE00037480068000C20F004013548006861F385
:104AF00012403349086048F248012046E26B904773
:104B00005AE06078401CC0B26070142810DD2C4858
:104B10000068000C20F004012948006861F312408D
:104B20002749086048F292012046E26B904743E033
:104B3000244800780A2808DA002060614FF47E409B
:104B400060814FF20100208503E0002060615A205F
:104B5000608131E06069401C6061282803D9002031
:104B60006061208D608127E000210846FFF732FE5A
:104B700013480068000C20F004011148006861F33C
:104B800012400F4908602046A16B884714E00021BD
:104B90000846FFF71FFE0A480068000C20F00401D9
:104BA0000748006861F312400549086048F2630154
:104BB0002046E26B904700BF00BF70BD6A0F002027
:104BC000480000208C0900200C000020F800002084
:104BD0000800002010B5044660895A2874D008DC0B
:104BE000012812D00A282DD014287ED01E286DD17D
:104BF00083E082286BD08C286AD0AA2869D0A0F5DF
:104C00007F40F0380028F2D12FE1AD4890F82C0019
:104C100000F0010080B1AB480068000C20F00401F6
:104C2000A848006861F31240A649086048F20C01E8
:104C30002046E26B904740E1A348406920610A208A
:104C400060813AE1A148007800F0080080B948F29C
:104C500091012046E26B90479A480068000C20F0D2
:104C600004019848006861F312409649086024E105
:104C7000954800780A2810DA92480068000C20F065
:104C800004019048006861F312408E49086048F2C0
:104C900092012046E26B90470FE18A4800780009B4
:104CA00000F00400B0B187480068000C20F0040157
:104CB0008448006861F312408249086048F2430169
:104CC0002046E26B9047F8E035E00EE0E0E03DE0A2
:104CD0007EE08EE07E48006840F010007C4908606D
:104CE0000020606114206081E7E06069401C606121
:104CF000282801D91E206081DFE07348007A0A2845
:104D000010DA70480068000C20F004016D4800685B
:104D100061F312406B49086048F248012046E26B9B
:104D20009047CAE06B4840896A4908820020E061E8
:104D30005A206081C1E04FF4207066494882822089
:104D4000608100210120FFF745FDB6E05E48406923
:104D50002169401AB0F5166F14D900210846FFF7F3
:104D600039FD58480068000C20F0040155480068DF
:104D700061F312405349086048F279012046E26B22
:104D800090479AE0504800780A2814DA0021084633
:104D9000FFF720FD4B480068000C20F00401494853
:104DA000006861F312404749086048F292012046CA
:104DB000E26B904781E04748407800B17DE00021F8
:104DC0000846FFF707FD002060618C20608174E0D9
:104DD0006069401C606128280AD9E069401CE061D4
:104DE000E069142802D3AA20608101E05A20608182
:104DF00063E03548007A0A2810DA32480068000C6F
:104E000020F004012F48006861F312402D4908602A
:104E100048F248012046E26B90474EE02D4A118A45
:104E20005089FEF797FA05280EDA26480068000C2C
:104E300020F004012348006861F312402149086012
:104E40002046A16B88470FE01E480068000C20F048
:104E500004011C48006861F312401A49086048F2D6
:104E6000B9012046E26B904727E000210846FFF792
:104E7000B1FC14480068000C20F0040111480068DF
:104E800061F312400F4908602046A16B884714E087
:104E900000210846FFF79EFC0A480068000C20F03D
:104EA00004010848006861F312400649086048F2AE
:104EB00063012046E26B904700BF00BF10BD0000B9
:104EC0006A0F0020480000208C0900200C00002000
:104ED00008000020F800002010B504466089B428BE
:104EE00075D008DC012813D00A282ED05A2875D096
:104EF0006E286ED17EE06FF470410844002869D0BE
:104F0000A0F6FF50002874D0B0F5F87FF1D1B6E0DC
:104F1000704890F82C0000F0010080B148F20C01BC
:104F20002046E26B90476C480068000C20F00401BA
:104F30006948006861F3124067490860C7E00020D3
:104F4000E061A0610A206081C1E06448007800F05F
:104F5000080080B960480068000C20F004015E4839
:104F6000006861F312405C49086048F291012046F4
:104F7000E26B9047ABE05A4800780A2810DA5648AE
:104F80000068000C20F004015348006861F31240EF
:104F90005149086048F292012046E26B904796E042
:104FA0004D480078000900F00400A0B14A480068AC
:104FB000000C20F004014848006861F312404649A3
:104FC000086048F243012046E26B90477FE01DE015
:104FD00004E067E036E05A20608178E041480068EC
:104FE00040F010003F490860002060616E20608141
:104FF0006DE03AE06069401C6061142805D9012128
:105000000846FFF7E7FBB420608160E03448007891
:105010000A280CDA00210846FFF7DCFB002060615B
:105020004FF47E4060814FF2010020854FE06069BF
:10503000401C6061142804D300206061A069401CFA
:10504000A06144E0E069401CE061254800780A283E
:1050500008DA002060614FF47E4060814FF2010069
:10506000208501E05A20608131E06069401C606168
:10507000282803D900206061208D608127E000216D
:105080000846FFF7A7FB14480068000C20F0040155
:105090001148006861F312400F4908602046A16B77
:1050A000884714E000210846FFF794FB0A4800688F
:1050B000000C20F004010848006861F31240064922
:1050C000086048F263012046E26B904700BF00BFD2
:1050D00010BD00006A0F0020480000200C000020D6
:1050E0008C0900200800002010B5044660891428AF
:1050F0002BD004DC01280AD00A2849D113E03B2830
:105100002ED0A0F57F40F038002841D13CE0244863
:10511000007800F0080010B10A20608102E020460B
:10512000A16B88473AE01F48407828B91E480068BC
:10513000000C00F0040028B148F246012046E26B62
:10514000904701E01420608128E01848006820F0B2
:10515000080016490860002060613B2060811DE066
:105160006069401C606128280DD92046A16B8847E2
:105170000D480068000C20F001010B48006861F345
:1051800012400949086009E02046A16B884705E004
:1051900048F265012046E26B904700BF00BF10BD9A
:1051A0000C000020F800002048000020080000202B
:1051B00010B5044660895A282ED004DC01280AD094
:1051C0000A284CD115E0BE2831D0A0F57F40F03838
:1051D000002844D13FE02648007800F0080018B1CC
:1051E0002046A16B884703E0002060610A206081AF
:1051F0003BE0204800780A2802DD5A20608134E034
:105200006069401C6061282805D948F29201204657
:10521000E26B904729E028E01748006840F008005A
:105220001549086000206061BE2060811DE0606952
:10523000401C60613C280DD92046A16B88470F486F
:105240000068000C40F001010C48006861F3124056
:105250000A49086009E02046A16B884705E048F24A
:1052600065012046E26B904700BF00BF10BD000003
:105270000C0000208C0900200800002048000020BD
:1052800010B5044660898C287DD00EDC64287BD064
:1052900006DC012821D00A2877D05A2876D1D3E01D
:1052A0006E2874D08228F9D16EE1B0F57E4F6FD0B0
:1052B00009DC96286DD097286CD06FF470410844B3
:1052C0000028EBD155E26FF47E410844002873D0EA
:1052D000A0F2EF100028E1D188E2FE4890F82C00FF
:1052E00000F0010080B1FC480068000C20F00401CF
:1052F000F948006861F31240F749086048F20C0170
:105300002046E26B904799E2F24890F82C0000F0BA
:10531000400080B1F0480068000C20F00401EE4825
:10532000006861F31240EC49086048F20A01204627
:10533000E26B904782E2206A002802DB206A132891
:1053400010DDE5480068000C20F00401E248006828
:1053500061F31240E049086048F209012046E26B1F
:1053600090476BE2DD48C0790A281CDDDC48C07834
:10537000216A884217D1D8480068000C20F0040147
:10538000D548006807E039E187E016E041E2EFE048
:1053900018E23EE18AE161F31240CF4908602046FD
:1053A000A16B88474AE2CD48406920610020207106
:1053B00060700A20608141E20EE2CA48007800F085
:1053C000080080B9C4480068000C20F00401C248FD
:1053D000006861F31240C049086048F2910120461C
:1053E000E26B90472AE2BD4800780A2810DABA48F2
:1053F0000068000C20F00401B748006861F3124017
:10540000B549086048F292012046E26B904715E2E8
:10541000B1480078000900F0040080B1AE4800688F
:10542000000C20F00401AC48006861F31240AA4966
:10543000086048F243012046E26B9047FEE10020FD
:1054400060615A206081F9E1A448007A0A280EDDE3
:10545000A54A236A12681C3232F81310A04A5089F8
:1054600000F052FE9E49488264206081E6E1606956
:10547000401C606128280FD997480068000C20F074
:1054800004019548006861F312409349086048F2AE
:1054900048012046E26B9047D0E19148B0F91200F4
:1054A000002833DA8E48408A404200B28C49488254
:1054B0000846B0F9120005280EDA87480068000C8B
:1054C00020F004018448006861F3124082490860BA
:1054D0002046A16B8847B1E18148B0F9120032281B
:1054E0000DDA7F48408A00F5207000B27C4948827E
:1054F0007E48006840F010007C49086033E07B483B
:10550000006820F01000794908602CE07448B0F978
:10551000120005280EDA70480068000C20F0040123
:105520006D48006861F312406B4908602046A16B2A
:10553000884783E16A48B0F9120032280DDA6848DA
:10554000408A00F5207000B26549488267480068CB
:1055500020F010006549086005E06448006840F0EC
:105560001000624908606E2060810020606165E182
:105570006069401C6061142805D900210120FFF7F3
:1055800029F98220608159E1544840692169401A13
:10559000B0F5966F14D900210846FFF71BF94E4865
:1055A0000068000C20F004014B48006861F31240D1
:1055B0004949086048F270012046E26B90473DE19E
:1055C000464800780A280CDA00210846FFF702F95D
:1055D000002060614FF47E4060814FF20100208521
:1055E0002CE13F48407800B128E100210846FFF750
:1055F000F1F80020A0618C2060811FE1A069401CAF
:10560000A061A0691E2803D90020A06196206081B6
:1056100014E13248007A0A2832DD334A236A1268DC
:105620001C3232F813102E4A5089FDF793FE0528DC
:1056300007DA002060614FF60160608197202085C5
:10564000FCE02079401CC0B22071052810DD224802
:105650000068000C20F004011F48006861F312404C
:105660001D49086048F2B0012046E26B9047E5E032
:10567000002060614FF47E4060815A202085DDE08B
:10568000A069401CA06150280FD913480068000C85
:1056900020F004011048006861F312400E490860D0
:1056A00048F248012046E26B9047C7E00B48007A79
:1056B0000A2848DD0C4A236A12681C3232F813109B
:1056C000074A5089FDF746FE05281DDA02480068A2
:1056D000000C0DE06A0F0020480000208C0900201B
:1056E000F80000200C0000200CCA00080800002070
:1056F00020F004015248006861F3124050490860EC
:105700002046A16B884799E02079401CC0B22071E7
:10571000052810DD4A480068000C20F004014848C4
:10572000006861F312404649086048F2B001204623
:10573000E26B904782E0002060614FF47E40608120
:105740005A2020857AE0A069401CA06150280FD91A
:105750003B480068000C20F004013948006861F300
:1057600012403749086048F248012046E26B9047F2
:1057700064E06078401CC0B26070142810DD3048CE
:105780000068000C20F004012D48006861F312400D
:105790002B49086048F292012046E26B90474DE0A9
:1057A000284800780A2808DA002060614FF47E401B
:1057B00060814FF20100208503E0002060615A20E3
:1057C00060813BE06069401C6061282803D90020AB
:1057D0006061208D608131E06069401C6061142847
:1057E00003D900206061208D608127E000210846F8
:1057F000FEF7F0FF12480068000C20F0040110488A
:10580000006861F312400E4908602046A16B88478A
:1058100014E000210846FEF7DDFF09480068000C8F
:1058200020F004010648006861F312400449086052
:1058300048F263012046E26B904700BF00BF10BDF5
:10584000480000208C09002010B5044660898C288F
:1058500074D00EDC642872D006DC012821D00A281E
:1058600056D05A286CD1AEE06E286AD08228F9D181
:1058700021E1B0F57E4F7AD009DC962878D09728C0
:1058800077D06FF4704108440028EBD10AE26FF43E
:105890007E41084400286DD0A0F2EF100028E1D12D
:1058A0003DE2F94890F82C0000F0010080B148F288
:1058B0000C012046E26B9047F4480068000C20F091
:1058C0000401F248006861F31240F04908604EE2BA
:1058D000ED4890F82C0000F0400080B1EB480068E3
:1058E000000C20F00401E948006861F31240E74928
:1058F000086048F20A012046E26B904737E2E4482C
:10590000406920610020207160700A2060812EE2D1
:10591000E048007800F00800A0B948F29101204664
:10592000E26B9047D9480068000C20F00401D7488A
:10593000006861F31240D549086018E2F5E06CE0B8
:1059400000E2ACE0D24800780A2814DACF480068B8
:10595000000C20F00401CD48006861F31240CB49EF
:10596000086048F292012046E26B9047FFE1C2E1F5
:10597000E6E033E1C9E1C5480078000900F0040021
:1059800080B1C2480068000C20F00401BF480068E4
:1059900061F31240BD49086048F243012046E26BC2
:1059A0009047E4E1BC48C07800F07F00401C14211F
:1059B00090FBF1F201FB1200B74908710020606111
:1059C0005A206081D3E1B248007A0A280FDDB24A3A
:1059D0001379B24A12681C3232F81310AE4A508959
:1059E00000F092FBAC49488264206081BFE16069AD
:1059F000401C606128280FD9A4480068000C20F0E2
:105A00000401A248006861F31240A049086048F20E
:105A100048012046E26B9047A9E19F48B0F9120087
:105A200000281EDA9C48408A404200B29A494882C7
:105A30000846B0F9120032280CDA0846408A00F510
:105A4000207000B248829648006840F010009449E7
:105A500008601FE09248006820F01000904908603C
:105A600018E08D48B0F9120032280DDA8A48408AD1
:105A700000F5207000B2884948828948006820F00B
:105A800010008749086005E08548006840F0100074
:105A9000834908606E2060810020606167E1606971
:105AA000401C6061142805D900210120FEF792FEF8
:105AB000822060815BE1764840692169401AB0F537
:105AC000966F14D900210846FEF784FE6F480068DF
:105AD000000C20F004016D48006861F312406B492E
:105AE000086048F270012046E26B90473FE1684849
:105AF00000780A280CDA00210846FEF76BFE002029
:105B000060614FF47E4060814FF2010020852EE1FC
:105B10006148407800B12AE100210846FEF75AFEAC
:105B20000020A0618C20608121E1A069401CA0615F
:105B3000A0691E2803D90020A0619620608116E18B
:105B40005348007A0A2833DD534A1379534A1268BE
:105B50001C3232F81310504A5089FDF7FBFB052820
:105B600007DA002060614FF6016060819720208590
:105B7000FDE02079401CC0B22071052810DD4348AB
:105B80000068000C20F004014048006861F31240F6
:105B90003E49086048F2B0012046E26B9047E6E0DB
:105BA000002060614FF47E4060815A202085DEE055
:105BB000A069401CA06150280FD934480068000C2F
:105BC00020F004013148006861F312402F49086059
:105BD00048F248012046E26B9047C8E02C48007A22
:105BE0000A283ADD2C4A13792C4A12681C3232F802
:105BF0001310294A5089FDF7ADFB05280EDA23481A
:105C00000068000C20F004012048006861F3124095
:105C10001E4908602046A16B8847A8E02079401CF7
:105C2000C0B22071052810DD18480068000C20F073
:105C300004011648006861F312401449086048F2F4
:105C4000B0012046E26B904791E0002060614FF484
:105C50007E4060815A20208589E0A069401CA061B7
:105C600050280FD909480068000C20F004010748AB
:105C7000006861F312400549086048F24801204677
:105C8000E26B904773E000006A0F0020480000209C
:105C90008C0900200C000020F80000200CCA00082D
:105CA000080000206078401CC0B26070142810DD2D
:105CB00030480068000C20F004012E48006861F3B1
:105CC00012402C49086048F292012046E26B90474E
:105CD0004DE0294800780A2808DA002060614FF476
:105CE0007E4060814FF20100208503E0002060616A
:105CF0005A2060813BE06069401C6061282803D91C
:105D000000206061208D608131E06069401C60612D
:105D1000142803D900206061208D608127E00021D4
:105D20000846FEF757FD13480068000C20F00401F8
:105D30001048006861F312400E4908602046A16BCC
:105D4000884714E000210846FEF744FD0948006832
:105D5000000C20F004010748006861F31240054977
:105D6000086048F263012046E26B904700BF00BF25
:105D700010BD0000480000208C0900207EB50346BD
:105D8000002206E0181D30F812002DF81200501CF9
:105D900082B2052AF6DB00221AE0002112E03DF86B
:105DA0001150481C3DF81000854209DD3DF81140B6
:105DB000481C3DF810002DF81100481C2DF810402B
:105DC000481C81B2C2F103008842E8DC501C82B258
:105DD000032AE2DBBDF80400BDF802502844BDF8F8
:105DE00006502844032590FBF5F080B27EBD0000EC
:105DF0002DE9F0410746B84600261420FDF79AFB2E
:105E0000002280213D4801F0DFF81420FDF792FBCD
:105E1000002426E008F0800028B101221021384833
:105E200001F0D2F804E000221021354801F0CCF84E
:105E30001420FDF77FFB01229103304801F0C4F8E4
:105E40001420FDF777FB00224FF480412B4801F02E
:105E5000BBF81420FDF76EFB4FEA48604FEA10686C
:105E6000641C082CD6D31420FDF764FB00221021FB
:105E7000234801F0A9F84FF4C870FDF75BFB01223D
:105E800091031E4801F0A0F81420FDF753FB0022F7
:105E90004FF48041194801F097F81420FDF74AFBB0
:105EA00000241DE001229103144801F08DF8142014
:105EB000FDF740FB4FF6FF7000EA460602210F484F
:105EC00001F076F805460DB146F0010600224FF4C8
:105ED00080410A4801F078F81420FDF72BFB641C80
:105EE000102CDFD301228021044801F06DF814202A
:105EF000FDF720FB3046BDE8F0810000000C0140BA
:105F0000001001402DE9F041002700BF781CC7B206
:105F100000224FF40051404801F056F800260022BC
:105F20004FF400413C4801F04FF80A20FDF702FB16
:105F300000251EE001225103374801F045F80F20EB
:105F4000FDF7F8FA00224FF40051334801F03CF815
:105F50000F20FDF7EFFA4FF6FF7000EA46064FF408
:105F600080512D4801F024F808B146F00106681C64
:105F7000C5B20C2DDEDB002400251EE001225103FA
:105F8000254801F021F80F20FDF7D4FA00224FF444
:105F90000051214801F018F80F20FDF7CBFA4FF619
:105FA000FF7000EA44044FF480511B4801F000F8F0
:105FB00008B144F00104681CC5B2062DDEDB0122E5
:105FC000D103154801F000F801225103124800F0F6
:105FD000FBFF304602F0EDFE04F00101884201D0E3
:105FE000032F93DB032F06DA0C48808D20F001008D
:105FF0000A4988850CE00948808D40F00100074976
:10600000888504F038044FF6FF7000EA84242643A4
:106010003046BDE8F0810000000C01406A0F00200E
:106020003548008800F4006028B13348006840F02B
:106030000040314908603048007800F0400048B125
:106040002E480078FF2808DA2C480078401C2B499D
:10605000087002E00020294908702748007800F005
:10606000800048B125484078FF2808DA2348407866
:10607000401C2249487002E0002020494870204816
:10608000006800F4803050B11E480078000940F0EC
:1060900004011C48006861F306101A49086016489C
:1060A000008800F4804098B114488079FF2804DA11
:1060B00012488079401C11498871104880790A285B
:1060C00009DD0D48006820F400400B49086002E03B
:1060D00000200A4988710A48008800F4804050B1C5
:1060E00008480088400B40F004010648006861F34E
:1060F0004F30044908607047040000208C090020DC
:106100000C000020480000202DE9F04706468A4692
:106110005546AD1BB5F5006F02DDA5F5805504E0D1
:1061200015F5006F01DA05F580555B4890F82C00F5
:1061300000F0400030B105EB8500C001CD2190FB9F
:10614000F1F5A6E04FF0000803E008F1010000F0CF
:10615000FF08524800681C3030F81800504502D043
:10616000B8F1140FF1DB3046FDF7F4FC00F07F04CA
:1061700004F11300142190FBF1F201FB1200C7B2ED
:10618000464800681C3030F81710444800681C303E
:1061900030F81400814219DA404800681C3030F8A9
:1061A0001700B04208DA3D4800681C3030F814008F
:1061B000B04201DDA14622E02746601C142190FB7D
:1061C000F1F201FB120000F0FF0918E0334800680B
:1061D0001C3030F81700B04206DB304800681C3035
:1061E00030F81400B04201DDA14608E02746601CEB
:1061F000142190FBF1F201FB120000F0FF09002DC9
:1062000022DD08F11400A0EB0900142190FBF1F24B
:1062100001FB1200C4B2214909681C3131F8191080
:1062200001F58051881BC11700EB11510913A0EB38
:10623000013505EB8500C001CD2190FBF1F504EBA4
:10624000840005EBC01524E0002D22DA07F11400CC
:10625000A0EB0800142190FBF1F201FB1200C4B284
:106260000E4909681C3131F8172006F58051881A4B
:10627000C11700EB11510913A0EB0135684200EB87
:106280008000C001CD2190FBF1F504EB8400A5EB6B
:10629000C01528B2BDE8F0876A0F00200CCA0008BC
:1062A0001FB50446002000900190029003906846BC
:1062B00000F096FE009818B9019808B9029808B144
:1062C000012000E0002010B9002004B010BD0098AB
:1062D00020800098C0F30F2060800198A080019872
:1062E000C0F30F20E080029820810298C0F30F20B5
:1062F00060810120E9E72DE9F04105460C4628467A
:10630000FFF776FD074621463846FAF725FA20467C
:10631000FFF734FD0746384602F072FD0646304668
:10632000BDE8F081F0B585B00621684602F010FBAB
:106330009DF803209DF8021002EB0120FAF78DF87A
:10634000064600220D4BFAF70BF80446FAF7EEF872
:106350000B4908609DF805209DF8041002EB012010
:10636000FAF77BF806460022044BF9F7F9FF0446DA
:10637000FAF7DCF80349086005B0F0BD00002440DE
:10638000380000203400002010B52C480068FAF7CF
:106390008DFE2A480068FAF74DFE28480068FAF793
:1063A0006DFD26480068FAF759FE24480068FAF7A0
:1063B000B9FE22480068FAF79DFD20480068FAF708
:1063C00061FE1E480068FAF7C1FE1C480068FAF733
:1063D0001DFE1A480068FAF705FE18480068FAF72B
:1063E00039FD16480068FAF7ADFD14480068FAF761
:1063F00095FD12480068FAF7E1FD10480068FAF7C9
:10640000C9FD0E480068FAF779FE0C480068FAF7F3
:1064100061FE0A480068FAF759FD08480068FAF773
:1064200041FD06480068FAF7B9FE04480068FAF72B
:10643000A1FE02480068FAF799FD10BD0C0000208B
:1064400070B50446002594F82100022803D00420EA
:10645000A0630125C1E02068006820F00E002168DB
:1064600008602068006820F00100216808605C492D
:106470002068884252D95A4978392068884201D127
:10648000012047E0564964392068884201D1102034
:1064900040E0534950392068884201D1801539E0E5
:1064A0004F493C392068884201D1801432E04C4980
:1064B00028392068884202D14FF480302AE04849C8
:1064C00014392068884202D14FF4801022E04449F8
:1064D0002068884201D140041CE04249206888427B
:1064E00001D1012016E03F4914312068884201D1D2
:1064F00010200FE03B4928312068884201D18015E7
:1065000008E038493C312068884201D1801401E01C
:106510004FF480303349091F086051E03049783921
:106520002068884201D1012047E02D496439206864
:10653000884201D1102040E0294950392068884222
:1065400001D1801539E026493C392068884201D1C3
:10655000801432E0224928392068884202D14FF461
:1065600080302AE01E4914392068884202D14FF455
:10657000801022E01A492068884201D140041CE0C2
:1065800018492068884201D1012016E015491431CC
:106590002068884201D110200FE01249283120687C
:1065A000884201D1801508E00E493C3120688842BC
:1065B00001D1801401E04FF48030094980394860EE
:1065C000012084F8210000BF002084F8200000BFD3
:1065D000606B10B12046616B8847284670BD000093
:1065E000800002400804024070B50446E06B056874
:1065F0002068066894F8401004208840284000284D
:1066000075D006F004000028FAD02068006800F079
:10661000200028B92068006820F004002168086084
:10662000D5492068884254D9D349783920688842AE
:1066300001D1042049E0D04964392068884201D161
:10664000402042E0CC4950392068884201D10015F1
:106650003BE0C9493C392068884202D14FF4804070
:1066600033E0C54928392068884202D14FF48020A0
:106670002BE0C14914392068884202D14FF48000D0
:1066800023E0BD492068884201D1C0041DE0BB4918
:106690002068884201D1042017E0B84914312068ED
:1066A000884201D1402010E0B44928312068884256
:1066B00001D1001509E0B1493C312068884202D17E
:1066C0004FF4804001E04FF48020AC49091F08607E
:1066D00054E0A94978392068884201D104204AE071
:1066E000A54964392068884202D1402043E04CE04B
:1066F000A14950392068884201D100153BE09E49EC
:106700003C392068884202D14FF4804033E09A49F6
:1067100028392068884202D14FF480202BE0964926
:1067200014392068884202D14FF4800023E0924956
:106730002068884201D1C0041DE090492068884249
:1067400001D1042017E08D4914312068884201D11D
:10675000402010E0894928312068884201D1001585
:1067600009E086493C312068884202D14FF48040DC
:1067700001E04FF48020804980394860E06A0028B9
:1067800002D02046E16A8847F4E094F840100220E5
:1067900088402840002871D006F002000028FAD076
:1067A0002068006800F0200040B92068006820F0F0
:1067B0000A0021680860012084F821006E492068E1
:1067C000884254D96C4978392068884201D1022026
:1067D00049E0694964392068884201D1202042E0BB
:1067E000654950392068884201D140153BE0624933
:1067F0003C392068884202D14FF4005033E05E49B2
:1068000028392068884202D14FF400302BE05A49E1
:1068100014392068884202D14FF4001023E0564911
:106820002068884201D180041DE0544920688842D4
:1068300001D1022017E0514914312068884201D16A
:10684000202010E04D4928312068884201D14015B0
:1068500009E04A493C312068884202D14FF4005097
:1068600001E04FF400304549091F086054E04249F7
:1068700078392068884202D102204AE057E03E4938
:1068800064392068884201D1202042E03A495039D9
:106890002068884201D140153BE037493C392068E7
:1068A000884202D14FF4005033E033492839206840
:1068B000884202D14FF400302BE02F491439206870
:1068C000884202D14FF4001023E02B49206888420F
:1068D00001D180041DE029492068884201D10220AD
:1068E00017E0264914312068884201D1202010E0A9
:1068F000224928312068884201D1401509E01F490A
:106900003C312068884202D14FF4005001E04FF43E
:10691000003019498039486000BF002084F8200009
:1069200000BFA06A30B32046A16A884722E094F8ED
:106930004010082088402840E0B106F00800C8B1A7
:106940002068006820F00E002168086094F840106C
:1069500001208840E16B48600120A06384F8210099
:1069600000BF002084F8200000BF206B10B120463B
:10697000216B884770BD000080000240080402407F
:106980000146002209B901207047204B086898424F
:106990000BD21F4B0868C01A1423B0FBF3F0800021
:1069A00008641B480838C8630AE0184B0868C01A16
:1069B0001423B0FBF3F08000086414480838C8635F
:1069C000022081F821000868026843F6F0708243D3
:1069D000D1E901031843CB6818430B6918434B698D
:1069E00018438B691843CB69184302430868026057
:1069F00000208862C862086348638863012081F8C8
:106A00002100002081F8200000BFBDE708040240FB
:106A1000080002402DE9F04104460D4616461F4687
:106A20004FF0000800BF94F82000012802D1022096
:106A3000BDE8F081012084F8200000BF94F8210017
:106A400001282CD1022084F821000020A0632068B6
:106A5000006820F00100216808603B463246294664
:106A60002046FCF7E3FCE06A30B12068006840F0A3
:106A70000E00216808600BE02068006820F0040028
:106A8000216808602068006840F00A0021680860FA
:106A90002068006840F001002168086006E000BF3F
:106AA000002084F8200000BF4FF002084046BFE7F6
:106AB00031B500F08FFA0546009C601C00B1641CE3
:106AC00000BF00F087FA401BA042FAD338BD000097
:106AD0002DE9F04104460E460127002500BF264857
:106AE000007E012802D10220BDE8F0810120224968
:106AF000087600BF2068022813D14CF25030FCF712
:106B0000D5FF90BB0120FCF757FF4CF25030FCF74B
:106B1000CDFF07461948006920F0040017490861B5
:106B200023E04CF25030FCF7C1FFF0B94FF0FF30DA
:106B30003060A56812E02846FCF752FF4CF2503056
:106B4000FCF7B4FF07460D48006920F002000B492E
:106B500008610FB1356007E005F50065D4E9021062
:106B600001EBC020A842E6D800BF00BF00200249C8
:106B7000087600BF3846B7E7A0000020002002409A
:106B80000348006940F08000014908610020704717
:106B9000002002402DE9FE4F05468B4617469846D9
:106BA000012600240020029000BF2448007E012816
:106BB00002D10220BDE8FE8F01202049087600BFE7
:106BC0004CF25030FCF772FF064686BB012D02D115
:106BD0000120029006E0022D02D10220029001E085
:106BE0000420029000241EE02201B946C246484615
:106BF0005146F9F7B9FA80B20190022000FB04B0C7
:106C000000900199FCF700FF4CF25030FCF74EFF6A
:106C100006460B48006920F001000949086106B1E9
:106C200004E0601CC4B202988442DDDB00BF00BFF8
:106C300000200249087600BF3046BBE7A0000020D4
:106C4000002002400748006900F0800028B1064893
:106C5000044948600548486001E001207047002071
:106C6000FCE700000020024023016745AB89EFCD1F
:106C70002DE9F8470246002400200025844600271D
:106C800000237BE14FF0010808FA03F4D1F80080FB
:106C900008EA0400A0427DD1DFF8ECA2D1F804801C
:106CA000A8EB0A09D0453AD014DCB8F1030F50D054
:106CB00009DCB8F1000F31D0B8F1010F1CD0B8F1E8
:106CC000020F49D120E0B8F1110F18D0B8F1120F1E
:106CD00042D11EE0B9F5881F25D006DCB9F5803F0A
:106CE00020D0B9F5801F37D11AE0B9F5001F18D0B0
:106CF000B9F5041F30D117E0D1F80CC02DE0D1F860
:106D00000C8008F1040C28E0D1F80C8008F1080C84
:106D100023E0D1F80C8008F10C0C1EE000BF00BF8E
:106D200000BF00BF00BF00BFD1F80880B8F1000F5E
:106D300002D14FF0040C0BE0D1F80880B8F1010F3C
:106D400003D14FF0080C146102E04FF0080C5461BD
:106D500003E04FF0000C00E000BF00BFFF2801D8A7
:106D6000904601E002F104084646FF2802D84FEAA7
:106D7000830803E0A3F108084FEA88084746D6F8DD
:106D800000804FF00F0909FA07F928EA09080CFA00
:106D900007F900E07AE048EA0908C6F80080D1F86F
:106DA000048008F08058B8F1805F6FD100BFDFF831
:106DB000DC81D8F8188048F00108DFF8D091C9F8D4
:106DC0001880C846D8F8188008F00108CDF800806F
:106DD00000BF00BF4FEAB9384FEA930958F829506D
:106DE0004FEA83784FEA18794FF00F0808FA09F84C
:106DF00025EA0805DFF89881424502D14FF00008E6
:106E000024E0DFF89081424502D14FF001081DE0F7
:106E1000DFF88481424502D14FF0020816E0DFF826
:106E20007C81424502D14FF003080FE0DFF870810A
:106E3000424502D14FF0040808E0DFF8688142457E
:106E400002D14FF0050801E04FF006084FEA8379C0
:106E50004FEA197908FA09F848EA0505DFF8488188
:106E60004FEA930948F82950D1F8048008F4803893
:106E7000B8F5803F0BD1DFF83481D8F8008048EABC
:106E80000008DFF82891C9F800800AE075E0DFF813
:106E90001C81D8F8008028EA0008DFF81091C9F8B2
:106EA0000080D1F8048008F40038B8F5003F0ED116
:106EB000DFF8F88008F10408D8F8008048EA0008F4
:106EC000DFF8E89009F10409C9F800800DE0DFF867
:106ED000DC8008F10408D8F8008028EA0008DFF810
:106EE000CC9009F10409C9F80080D1F8048008F4B5
:106EF0008018B8F5801F0ED1DFF8B08008F10808BF
:106F0000D8F8008048EA0008DFF8A09009F10809E5
:106F1000C9F800800DE0DFF8948008F10808D8F87F
:106F2000008028EA0008DFF8849009F10809C9F810
:106F30000080D1F8048008F40018B8F5001F0ED1C5
:106F4000DFF8688008F10C08D8F8008048EA0008EB
:106F5000DFF8589009F10C09C9F800800DE0DFF85E
:106F60004C8008F10C08D8F8008028EA0008DFF807
:106F70003C9009F10C09C9F800805B1C102BFFF450
:106F800081AEBDE8F887000000001110001002403B
:106F900000080140000C01400010014000140140B5
:106FA00000180140001C014008000140000401409D
:106FB000024693680B400BB1012000E000207047AF
:106FC000C2684A40C26070470AB1016101E00B0427
:106FD000036170470148006870470000000000200E
:106FE0000549096801600449091D096841600249B1
:106FF0000831096881607047E8F7FF1F02480068A0
:10700000401C0149086070470000002010B5084886
:10701000006840F0100006490860032000F0BCF84A
:10702000002000F007F800F019F8002010BD000063
:107030000020024070B50446074800684FF47A719A
:10704000B0FBF1F5284600F0CCFC00222146501E92
:1070500000F063F8002070BD9400002008B500BF68
:107060002548806940F0010023498861084680690D
:1070700000F00100009000BF00BF032000F08CF87A
:10708000002211466FF00B0000F047F80022114675
:107090006FF00A0000F041F8002211466FF009007D
:1070A00000F03BF800221146501F00F036F8002295
:1070B0001146101F00F031F800221146901E00F01A
:1070C0002CF800221146501E00F027F8002211462D
:1070D000052000F022F8052000F012F800BF074854
:1070E000406820F0E060054948600846406840F08C
:1070F0008060486000BF08BD0010024000000140F1
:1071000000BF00F01F02012191404209920002F1EC
:10711000E022C2F8001100BF70472DE9F05F804601
:107120000D461646002702F0F3FB074639462A466D
:10713000334601F00700C0F1070ABAF1040F02D983
:107140004FF0040A01E0C0F1070AD14600F1040A39
:10715000BAF1070F02D24FF0000A01E0A0F1030AD2
:10716000D4464FF0010A0AFA09FAAAF1010A0AEA1A
:10717000020A0AFA0CFA4FF0010B0BFA0CFBABF106
:10718000010B0BEA030B4AEA0B042146404602F0CE
:10719000C7FBBDE8F09F000000BF00F00702064BF0
:1071A00019684FF6FF031940044B0B4343EA0221D1
:1071B000014B196000BF70470CED00E00000FA05BC
:1071C000F8B5044600260025207800F001000028CC
:1071D0006BD000274348C06900F0805070B900BFF1
:1071E0004048C06940F080503E49C8610846C069C7
:1071F00000F08050009000BF00BF01273A480068AF
:1072000000F48070B0B93848006840F480703649A6
:107210000860FFF7DFFE064606E0FFF7DBFE801B97
:10722000642801D90320F8BD2F48006800F480705D
:107230000028F2D02B48006A00F440752DB3A088D6
:1072400000F44070A84220D02648006A20F440751F
:10725000012026490860002008602248056205F0E8
:10726000010090B1FFF7B6FE064608E0FFF7B2FE58
:10727000801B41F28831884201D90320D3E71948A5
:10728000006A00F002000028F0D01648006A20F4DE
:1072900040706168084313490862012F04D1084611
:1072A000C06920F08050C86100BF207800F0020063
:1072B000022807D10B48406820F44040A1680843E9
:1072C00008494860207800F01000102807D10548D0
:1072D000406820F48000616908430249486000204A
:1072E000A1E700000010024000700040400442424C
:1072F00070B504460D4600266248006800F007009D
:10730000A8420ED25F48006820F0070028435D497C
:1073100008600846006800F00700A84201D001207C
:1073200070BD207800F00200022807D1564840685E
:1073300020F0F000A168084353494860207800F02D
:10734000010000285DD06068012806D14E48006821
:1073500000F4003090B90120E2E76068022806D10D
:107360004948006800F0007040B90120D8E746485D
:10737000006800F0020008B90120D1E742484068E7
:1073800020F00300616808433F494860FFF722FE90
:1073900006466068012810D108E0FFF71BFE801B3D
:1073A00041F28831884201D90320B9E73648406864
:1073B00000F00C000428F0D123E06068022810D10E
:1073C00008E0FFF707FE801B41F28831884201D9AF
:1073D0000320A5E72C48406800F00C000828F0D1F5
:1073E0000FE008E0FFF7F6FD801B41F2883188428C
:1073F00001D9032094E72448406800F00C000028DD
:10740000F0D12048006800F00700A8420ED91D48BE
:10741000006820F0070028431A4908600846006801
:1074200000F00700A84201D0012079E7207800F0A1
:107430000400042807D11448406820F4E060E168A3
:10744000084311494860207800F00800082808D156
:107450000D48406820F46050216940EAC1000A49A3
:10746000486000F03DF808494968C1F30311074A34
:10747000515CC840064908600020FFF7DBFD002092
:107480004EE70000002002400010024014CA00082D
:10749000940000200148006870470000940000201C
:1074A00000B5FFF7F7FF04494968C1F30221034A19
:1074B000515CC84000BD00000010024024CA000812
:1074C00000B5FFF7E7FF04494968C1F3C221034A49
:1074D000515CC84000BD00000010024024CA0008F2
:1074E000F0B585B00FF2700C9CE8E01001A8A0E8A0
:1074F000E0101DA52D680095002100240022002326
:1075000000201A4D696801F00C05FDB1042D02D070
:10751000082D1AD101E016481AE001ADC1F38346E7
:10752000AB5D01F480355DB1104D6D68C5F340452C
:107530001DF805400E4DB5FBF4F505FB03F202E026
:107540000C4D03FB05F2104602E000BF084800BFE7
:1075500000BF05B0F0BD00000203040506070809DE
:107560000A0B0C0D0E0F101001020000001002405B
:1075700000127A0000093D00F8B504460025207885
:1075800000F00100002878D0F848406800F00C00B6
:1075900004280CD0F548406800F00C00082811D1F0
:1075A000F248406800F48030B0F5803F0AD1EF48DF
:1075B000006800F4003000285FD0606800285CD1CB
:1075C0000120F8BD00BF6068B0F5803F06D1E748F4
:1075D000006840F48030E549086028E0606858B9E8
:1075E000E248006820F48030E049086008460068FE
:1075F00020F4802008601AE06068B0F5A02F0BD15D
:10760000DA48006840F48020D849086008460068DD
:1076100040F4803008600AE0D448006820F48030EC
:10762000D24908600846006820F48020086000BF46
:10763000606888B1FFF7CEFC054606E0FFF7CAFC9C
:10764000401B642801D90320BBE7C848006800F448
:1076500000300028F2D010E0FFF7BCFC054606E041
:10766000FFF7B8FC401B642801D90320A9E7BF48F5
:10767000006800F400300028F2D1207800F0020009
:10768000022857D1B948406800F00C0050B1B74803
:10769000406800F00C00082818D1B448406800F495
:1076A000803098B9B148006800F0020020B120692C
:1076B000012801D0012084E7AC48006820F0F800E0
:1076C000616940EAC100A949086033E02069E8B176
:1076D0000120A7490860FFF77DFC054606E0FFF79B
:1076E00079FC401B022801D903206AE79F48006803
:1076F00000F002000028F2D09C48006820F0F8005A
:10770000616940EAC1009949086013E00020984986
:107710000860FFF75FFC054606E0FFF75BFC401BD7
:10772000022801D903204CE79048006800F00200CD
:107730000028F2D1207800F0080008282DD1A06997
:10774000B8B101208B490860FFF744FC054606E00C
:10775000FFF740FC401B022801D9032031E7834892
:10776000406A00F002000028F2D0012002F05EF929
:1077700013E000207F490860FFF72CFC054606E077
:10778000FFF728FC401B022801D9032019E777489E
:10779000406A00F002000028F2D1207800F00400D6
:1077A000042873D100267148C06900F0805070B978
:1077B00000BF6E48C06940F080506C49C8610846FF
:1077C000C06900F08050009000BF00BF01266A48E9
:1077D000006800F48070B0B96748006840F48070B9
:1077E00065490860FFF7F6FB054606E0FFF7F2FB88
:1077F000401B642801D90320E3E65F48006800F4D9
:1078000080700028F2D000BFE068012806D15748F8
:10781000006A40F001005549086227E0E06858B965
:107820005248006A20F00100504908620846006A88
:1078300020F00400086219E0E06805280BD14B48ED
:10784000006A40F00400494908620846006A40F0B6
:10785000010008620AE04548006A20F0010043493F
:1078600008620846006A20F00400086200BFE06871
:10787000A0B1FFF7AFFB054609E0FFF7ABFB401BEC
:1078800041F28831884202D903209AE622E0374843
:10789000006A00F002000028EFD012E0FFF79AFB28
:1078A000054608E0FFF796FB401B41F2883188420D
:1078B00001D9032085E62D48006A00F00200002867
:1078C000F0D1012E05D12948C06920F08050274908
:1078D000C86100BFE069C8B32448406800F00C00EC
:1078E000082860D0E069022848D1002020490866B5
:1078F000FFF770FB054606E0FFF76CFB401B022814
:1079000001D903205DE61948006800F000700028E6
:10791000F2D1206AB0F5803F07D11448406820F4C6
:107920000030A168084311494860D4E908010843C0
:107930000E49496821F4741108430C49486001203C
:107940000B490866FFF746FB054607E02DE0FFF709
:1079500041FB401B022801D9032032E6034800689E
:1079600000F000700028F2D01FE00000001002407C
:1079700000004242800442420070004000200C4956
:107980000866FFF727FB054606E0FFF723FB401BD1
:10799000022801D9032014E60648006800F00070B0
:1079A0000028F2D101E001200BE6002009E60000EA
:1079B0000000424200100240042808D14FF0E021AC
:1079C000096941F004014FF0E022116107E04FF036
:1079D000E021096921F004014FF0E02211617047B4
:1079E000704770B504462546681EB0F1807F01D30C
:1079F00001200FE0681E4FF0E02148610F214FF099
:107A0000FF3001F08DFF00204FF0E021886107205A
:107A10000861002070BD10B5FFF7E2FF10BD704790
:107A2000704710B50346002200BF93F83C000128C0
:107A300001D1022010BD012083F83C0000BF22F0DC
:107A4000FF00CC6840EA040222F440708C6840EAEF
:107A5000040222F480604C6840EA040222F40060D0
:107A60000C6840EA040222F480500C6940EA0402E7
:107A700022F400504C6940EA040222F480408C69F0
:107A800040EA040222F400408C6940EA04021868CB
:107A9000426400BF002083F83C0000BF00BFC9E77C
:107AA000024600BF92F83C00012801D10220704735
:107AB000012082F83C0000BF022082F83D001068DF
:107AC000406820F0700013685860106840680B68C8
:107AD0001843136858601068806820F080001368AD
:107AE0009860106880684B6818431368986001209C
:107AF00082F83D0000BF002082F83C0000BF00BFBC
:107B0000D5E710B504460CB9012010BD94F83D002E
:107B100028B9002084F83C00204600F00DF802202F
:107B200084F83D00211D206803F03CF8012084F812
:107B30003D000020E9E7000038B504461A492068F6
:107B400088420DD100BF1948C06940F004001749B0
:107B5000C8610846C06900F00400009000BF21E041
:107B60001349206888421DD100BF1048806940F445
:107B700000500E4988610846806900F4005000906A
:107B800000BF00BF002211462C20FFF7C6FA2C20B0
:107B9000FFF7B6FA06480C30006840F001000449CF
:107BA0000C31086038BD00000008004000100240A1
:107BB000003401402DE9F04104460D46002600BF87
:107BC00094F83C00012802D10220BDE8F081012098
:107BD00084F83C0000BF022084F83D0020688668DD
:107BE00026F0770626F47F462068866028685028AD
:107BF0003BD00CDC202860D004DC002853D01028B7
:107C000065D155E030285DD0402860D141E0602842
:107C100035D070280DD0B0F5805F03D0B0F5005F8F
:107C200055D115E02068806820F007002168886041
:107C30004EE0D5E902136A68206803F00DF8206869
:107C4000866826F0770646F07706206886603FE073
:107C5000D5E902136A68206802F0FEFF2068806898
:107C600040F480402168886032E0EA6869682068F2
:107C700003F0F0F85021206802F0FAFF28E0EA68EB
:107C80006968206803F0FBF86021206802F0F0FFCB
:107C90001EE0EA686968206803F0DCF8402120688B
:107CA00002F0E6FF14E00021206802F0E1FF0FE09F
:107CB0001021206802F0DCFF0AE02021206802F099
:107CC000D7FF05E03021206802F0D2FF00E000BFBE
:107CD00000BF012084F83D0000BF002084F83C0074
:107CE00000BF00BF71E7704710B504462068006907
:107CF000C0F34000D8B12068C068C0F34000B0B104
:107D00006FF00200216808610120207720688069F7
:107D100000F0030018B12046FFF7E5FF05E020461C
:107D200000F018F9204600F0D0F9002020772068F4
:107D30000069C0F38000D8B12068C068C0F380003B
:107D4000B0B16FF00400216808610220207720683C
:107D5000806900F4407018B12046FFF7C4FF05E0C9
:107D6000204600F0F7F8204600F0AFF90020207719
:107D700020680069C0F3C000D8B12068C068C0F3B3
:107D8000C000B0B16FF008002168086104202077BE
:107D90002068C06900F0030018B12046FFF7A3FF78
:107DA00005E0204600F0D6F8204600F08EF90020CD
:107DB000207720680069C0F30010D8B12068C0683F
:107DC000C0F30010B0B16FF0100021680861082006
:107DD00020772068C06900F4407018B12046FFF792
:107DE00082FF05E0204600F0B5F8204600F06DF96E
:107DF000002020772068006900F0010058B1206859
:107E0000C06800F0010030B16FF001002168086126
:107E1000204600F0C5F920680069C0F3C01058B1D1
:107E20002068C068C0F3C01030B16FF080002168D6
:107E300008612046FFF7F3FD20680069C0F3801059
:107E400058B12068C068C0F3801030B16FF04000B6
:107E500021680861204600F0A4F920680069C0F399
:107E6000401058B12068C068C0F3401030B16FF0C6
:107E70002000216808612046FFF7D2FD10BD0000F8
:107E80001FB5044611492068884210D18014009023
:107E9000022001900320039069460D48FEF7E8FE9A
:107EA0000C48406840F480500A4948600CE00A4998
:107EB0002068884208D14020009002200190039061
:107EC00069460648FEF7D4FE1FBD000000080040CA
:107ED0000014014000000140003401400010014046
:107EE00070B504460E46154600BF94F83C000128C4
:107EF00001D1022070BD012084F83C0000BF0220A7
:107F000084F83D0035B1042D09D0082D0CD00C2D7E
:107F100014D10EE03146206802F0B4FE0FE0314685
:107F2000206802F0EBFE0AE03146206802F026FFEE
:107F300005E03146206802F061FF00E000BF00BFAD
:107F4000012084F83D0000BF002084F83C0000BF01
:107F500000BFCFE7704710B504460CB9012010BD33
:107F600094F83D0028B9002084F83C00204600F039
:107F70000CF8022084F83D00211D206802F012FE5A
:107F8000012084F83D000020E9E7704770B5044601
:107F90000D46164600BF94F83C00012801D102208E
:107FA00070BD012084F83C0000BF022084F83D0031
:107FB00036B1042E1BD0082E31D00C2E5ED145E0F8
:107FC0002946206802F05EFE2068806940F00800C3
:107FD000216888612068806920F004002168886138
:107FE00020688069296908432168886147E029463B
:107FF000206802F083FE2068806940F400602168F8
:1080000088612068806920F4806021688861206828
:108010008069296940EA0120216888612FE02946AA
:10802000206802F0ABFE2068C06940F008002168BB
:10803000C8612068C06920F004002168C861206818
:10804000C069296908432168C86118E02946206889
:1080500002F0D4FE2068C06940F400602168C86165
:108060002068C06920F480602168C8612068C06908
:10807000296940EA01202168C86100E000BF00BF13
:10808000012084F83D0000BF002084F83C0000BFC0
:1080900000BF85E710B504460CB9012010BD94F867
:1080A0003D0028B9002084F83C00204600F00CF880
:1080B000022084F83D00211D206802F073FD01209C
:1080C00084F83D000020E9E77047704730B504466A
:1080D0000D4601222946206802F0B0FD0C492068B7
:1080E000884203D00B492068884201D1012000E07A
:1080F000002028B12068406C40F4004021684864AA
:108100002068006840F0010021680860002030BD50
:10811000002C01400034014030B504460D460022D9
:108120002946206802F08AFD1B492068884203D056
:108130001A492068884201D1012000E0002090B156
:1081400000BF2068006A41F21111084050B9206850
:10815000006A8910084028B92068406C20F400406B
:108160002168486400BF00BF2068006A41F2111115
:10817000084050B92068006A8910084028B9206872
:10818000006820F001002168086000BF012084F829
:108190003D00002030BD0000002C014000340140B3
:1081A00070477047704700002DE9F047044620688B
:1081B00005682068C668206847694FF00008C14616
:1081C00005F00F08B8F1000F0AD105F0200038B112
:1081D00006F0200020B1204603F004F8BDE8F08747
:1081E000B8F1000F6DD007F0010018B906F49070D7
:1081F000002866D005F0010030B106F4807018B197
:10820000E06B40F00100E06305F0040030B107F0DE
:10821000010018B1E06B40F00200E06305F00200DD
:1082200030B107F0010018B1E06B40F00400E063EA
:1082300005F0080030B107F0010018B1E06B40F024
:108240000800E063E06B68B305F0200028B106F099
:10825000200010B1204602F0C5FF20684069C0F33D
:108260008019E06B00F0080010B9B9F1000F22D0BE
:10827000204602F08DFF2068406900F04000B0B158
:108280002068406920F0400021684861606B50B16F
:108290001748616B4863606BFEF7D2F810B1606BF2
:1082A000416B88470CE02046FFF77CFF08E0204642
:1082B000FFF778FF04E02046FFF774FF0020E0633B
:1082C0008CE705F0800030B106F0800018B1204640
:1082D00003F0C0F882E705F0400030B106F040003E
:1082E00018B1204602F064FF78E700BF76E700008F
:1082F00095B0000810B504460CB9012010BDA06966
:1083000000B100E000BF94F8390028B9002084F8DB
:108310003800204600F028F8242084F8390020682E
:10832000C06820F400502168C860204602F0AEFF0B
:108330002068006920F49040216808612068406945
:1083400020F02A00216848612068C06840F400508D
:108350002168C8600020E063202084F8390084F898
:108360003A000020CAE7000010B586B00446CF49A5
:108370002068884260D100BFCD48C06940F4002029
:10838000CB49C8610846C06900F40020019000BFD5
:1083900000BF08150290022003900320059002A957
:1083A000C448FEF765FC4FF4006002900020039083
:1083B000049002A9BF48FEF75BFCBF48BF490860B4
:1083C000002048600021BD4881608021C1600021FB
:1083D000016141618161C161FEF7D2FA20B140F2D1
:1083E0003711B7A003F0AEF900BFB4486063446230
:1083F00000BFB1482830B64908601020486000210D
:10840000B34881608021C1600021016141618161C7
:10841000C161FEF7B5FA20B140F24711A8A003F000
:1084200091F900BFAA482063446200BF00221146B0
:108430003420FEF772FE37E1A6492068884263D1F6
:1084400000BF9B48806940F4804099498861084694
:10845000806900F48040019000BF00BF4815029081
:10846000022003900320059002A99B48FEF700FC20
:108470004FF48060029000200390049002A9964877
:10848000FEF7F6FB954896490860002048600021F9
:10849000934881608021C160002101614161816157
:1084A000C161FEF76DFA20B140F2751184A003F0AE
:1084B00049F900BF8A486063446200BF87481438A6
:1084C000884908601020486000218648816080212A
:1084D000C1600021016141618161C161FEF750FA13
:1084E00020B140F2851176A003F02CF900BF7D4841
:1084F0002063446200BF002211462520FEF70DFED6
:108500002520FEF7FDFDCFE077492068884263D142
:1085100000BF6748C06940F400306549C86108463B
:10852000C06900F40030019000BF00BF0420029039
:10853000022003900320059002A96748FEF798FBEC
:108540000820029000200390049002A96248FEF7E0
:108550008FFB6248143065490860002048600021A4
:10856000624881608021C1600021016141618161B7
:10857000C161FEF705FA20B140F2B31150A003F03B
:10858000E1F800BF59486063446200BF5348283097
:1085900057490860102048600021554881608021BB
:1085A000C1600021016141618161C161FEF7E8F9AB
:1085B00020B140F2C31142A003F0C4F800BF4C4800
:1085C0002063446200BF002211462620FEF7A5FD6D
:1085D0002620FEF795FD67E046492068884263D172
:1085E00000BF3348C06940F480203149C861084663
:1085F000C06900F48020019000BF00BF0815029000
:10860000022003900320059002A93B48FEF730FBAF
:108610004FF40060029000200390049002A93648B5
:10862000FEF726FB2D483C3834490860102048608E
:108630000021324881608021C160002101614161D7
:108640008161C161FEF79CF920B140F2F1111CA0DB
:1086500003F078F800BF29482063446200BF1F4838
:10866000283827490860002048600021244881609C
:108670008021C1600021016141618161C161FEF71A
:108680007FF920B140F201210DA003F05BF800BF9B
:108690001B486063446200BF002211462720FEF79A
:1086A0003CFD2720FEF72CFD06B010BD004C00401D
:1086B0000010024000100140300402406C0700200E
:1086C0002E2E2F5372632F75736172742E63000008
:1086D000B007002000380140000801405800024067
:1086E000F407002038080020004400407C080020E7
:1086F000C008002000480040000C01400409002090
:108700004809002077B581B00446154694F83A0030
:10871000202850D1029800B115B9012004B070BDD5
:1087200000BF94F83800012801D10220F6E70120AB
:1087300084F8380000BF0298A062A5850020E0639D
:10874000222084F83A001D48616B88621C48616BE6
:10875000C8621C48616B08630020616B486302AE0D
:1087600032682368191D2B46606BFEF753F900BF72
:108770000020009020680068009020684068009009
:1087800000BF00BF00BF002084F8380000BF206891
:10879000C06840F480702168C8602068406940F07B
:1087A0000100216848612068406940F0400021686C
:1087B00048610020B2E70220B0E70000F9B00008ED
:1087C0003FB10008A9B0000870477047F7B50446EC
:1087D000154694F8390020283DD1019800B10DB913
:1087E0000120FEBD00BF94F83800012801D102200D
:1087F000F7E7012084F8380000BF01982062A584C3
:10880000E5840020E063212084F839001348216BBF
:1088100088621348216BC8621248216B08630020EC
:10882000216B486301AE23681A1D31682B46206B0B
:10883000FEF7F0F86FF040002168086000BF0020EC
:1088400084F8380000BF2068406940F0800021684B
:1088500048610020C5E70220C3E700004DB10008D1
:1088600083B10008A9B00008134909680268914261
:1088700008D10121114A51720168496941F0800112
:10888000026851610E4909680268914202D10121D2
:108890000C4A51720C4909680268914202D10121C7
:1088A0000A4A51720A4909680268914202D10121BB
:1088B000084A517270470000AC060020F801002001
:1088C000EC060020220500202C0700209005002047
:1088D0006C060020FE050020704700BFFEE7000088
:1088E00070B5184890F82D0070B1164890F82D001A
:1088F000401E40B2134981F82D001348006840F033
:1089000000701149086005E00F48006820F0007011
:108910000D4908600B498869F7F7DDFD0446002220
:108920000A4BF7F7EBFD06D20748006840F080607D
:108930000549086005E00448006820F080600249AD
:10894000086070BD2C010020080000200000694074
:1089500070B505460C4600F01BF9B826304600F00D
:10896000D7F800F06FF94FF47A70FAF7E9FD00F0EC
:108970003DF900F00DF900BF304600F0C9F800F0F5
:1089800061F9032000F0C4F800F05CF9002000F069
:10899000BFF800F057F9042000F0BAF800F052F9DF
:1089A00000F024F941F27070FAF7CAFD00F0F0F817
:1089B000B926304600F0ACF800F044F93220FAF75E
:1089C000BFFD0CE000F068F82870012C02D100F027
:1089D00037F801E000F008F86D1C601EC4B2002CEE
:1089E000F0D100F003F970BD1FB500224FF48051A3
:1089F0001248FEF7E9FA4FF4006000900120019060
:108A00000320039069460D48FEF732F900224FF427
:108A100000610A48FEF7D8FA2820FAF791FD0122F2
:108A200011030648FEF7D0FA2820FAF789FD002244
:108A30004FF480510148FEF7C7FA1FBD00080140FE
:108A40001FB500224FF480511248FEF7BDFA4FF4D3
:108A500000600090012001900320039069460D48BA
:108A6000FEF706F90122D1020A48FEF7ADFA2820E6
:108A7000FAF766FD012211030648FEF7A5FA282041
:108A8000FAF75EFD00224FF480510248FEF79CFA8F
:108A90001FBD0000000801407FB500244FF40060B6
:108AA0000090002001900120029069461748FEF7CF
:108AB000DFF8002525E000224FF480511348FEF72F
:108AC00083FA3220FAF73CFD012211030F48FEF72A
:108AD0007BFA3220FAF734FD6006040E4FF4006191
:108AE0000A48FEF765FA08B144F001043220FAF7AB
:108AF00027FD00224FF480510448FEF765FA681CF8
:108B0000C5B2082DD7DB204604B070BD0008014077
:108B10007FB504464FF400600090012001900320CF
:108B2000039069461948FEF7A3F800224FF48051DC
:108B30001648FEF749FA002525E0E00928B1012290
:108B4000D1021248FEF740FA05E000224FF400611E
:108B50000E48FEF739FA6006040E3220FAF7F0FCF0
:108B6000012211030948FEF72FFA3220FAF7E8FC38
:108B700000224FF480510548FEF726FA3220FAF71A
:108B8000DFFC681CC5B2082DD7DB7FBD00080140A3
:108B90001FB54FF400600090012001900320039066
:108BA00069461148FEF764F80122D1020E48FEF72B
:108BB0000BFA012211030C48FEF706FA3220FAF7ED
:108BC000BFFC00224FF400610748FEF7FDF9322098
:108BD000FAF7B6FC00224FF480510348FEF7F4F98F
:108BE0003220FAF7ADFC1FBD000801401FB54FF45D
:108BF0000060009001200190032003906946104816
:108C0000FEF736F800224FF480510D48FEF7DCF9EC
:108C100000224FF400610A48FEF7D6F93220FAF735
:108C20008FFC012211030648FEF7CEF90122D10282
:108C30000348FEF7C9F93220FAF782FC1FBD000095
:108C4000000801401FB500240122D1021748FEF799
:108C5000BBF92820FAF774FC4FF400600090002064
:108C600001900120029069461048FEF701F80122A8
:108C700011030E48FEF7A8F92820FAF761FC06E078
:108C8000601CC4B2FA2C02DD002004B010BD4FF409
:108C900000610648FEF78CF90028F1D100224FF45C
:108CA00080510248FEF790F90120EEE700080140EC
:108CB0004FF6FF71C18041810021C18100F128017F
:108CC000416300210162044901630449C16204490E
:108CD00081630449C1637047D80900203C0F00201C
:108CE000E5A8000861A800083C22B1FBF2F302FBF2
:108CF000131282723C22B1FBF2F1B1FBF2F302FBE0
:108D0000131242723C22B1FBF2F11822B1FBF2F3D2
:108D100002FB1312027270472DE9F04104464FF036
:108D20008141A068F7F7DEFA07464FF0814061689D
:108D3000F7F7D8FA80464FF07E51F7F749FA064622
:108D40003946F7F745FA05462168F7F799FAE061E1
:108D50004FF08040A168F7F793FA07464FF0814142
:108D6000F7F7C0FA06464FF07E51F7F731FA05469D
:108D70002168F7F785FA2062A1682068F7F780FA82
:108D800005464FF08141F7F7ADFA6062002020619F
:108D90006061E06084F82C0084F82D00BDE8F0816B
:108DA000002101614161C16080F82C1080F82D1014
:108DB0007047014681EA212181EA211181EAA1015E
:108DC00081EA610101F0010008B1002100E0012108
:108DD000C8B2704701464FF4C87091FBF0F300FB36
:108DE000131040B10A46C81701EB90708010A1EB38
:108DF000800010B909B1012070470020FCE7000095
:108E00002DE9F84F05460026002700248648006813
:108E1000807800287ED04FF6F070854201DD834EC9
:108E2000FEE08348006800F023FE07462846F7F777
:108E30000FFB80467F49F7F723FA0646394630464E
:108E4000F7F7C6F9064601E0601CC4B27A4850F84C
:108E500024103046F7F790FB01D2822CF4DD621E1D
:108E6000754B53F822101A4652F82400F7F702FA0D
:108E700083467249F7F736FA8146601E6E4A52F809
:108E800020103046F7F7F6F982464946F7F72AFAF6
:108E90008046611E01EB81014800F7F7D0FA414698
:108EA0000090F7F795F906465F480068408940F260
:108EB000DC51884213DA5C4800684089B0F5FA7FDB
:108EC0000DDD594909684889F7F7C2FA81463146EC
:108ED000F7F7D6F980465A49F7F704FA0646594992
:108EE0003046F7F73FFB9BD24F480068B0F90C00C3
:108EF000642895DA4C480068B0F90C0010F1640F52
:108F00008EDD49490968B1F90C00F7F798FA8046F7
:108F1000314600E003E0F7F75BF9064680E04FF6E4
:108F2000F070854201DD484E7AE04148006800F06B
:108F30009FFD07462846F7F78BFA80464349F7F727
:108F40009FF9064639463046F7F742F9064601E0F2
:108F5000601CC4B2384850F824103046F7F70CFBB8
:108F600001D2822CF4DD621E334B53F822101A46D4
:108F700052F82400F7F77EF983463049F7F7B2F943
:108F80008146601E2C4A52F820103046F7F772F9DD
:108F900082464946F7F7A6F98046611E01EB81013A
:108FA0004800F7F74CFA41460090F7F711F90646EA
:108FB0001D480068408940F2DC51884213DA1A48A3
:108FC00000684089B0F5FA7F0DDD174909684889C6
:108FD000F7F73EFA81463146F7F752F980461849CD
:108FE000F7F780F9064617493046F7F7BBFA17D26C
:108FF0000D480068B0F90C00642811DA0A480068CE
:10900000B0F90C0010F1640F0ADD07490968B1F9E5
:109010000C00F7F714FA80463146F7F7D9F8064600
:109020003046BDE8F88F00000CCA000800E0954407
:10903000340000201905463AE0C300080000204132
:1090400000007A440000964300C07944E3BA1E3A17
:1090500008B500BF2D48406940F001002B49486128
:109060000846406900F00100009000BF00BF00BF4B
:109070000846406940F0020048610846406900F037
:109080000200009000BF00BF002211460C20FEF736
:1090900044F80C20FEF734F8002211460D20FEF7AC
:1090A0003CF80D20FEF72CF8002211460E20FEF7AA
:1090B00034F80E20FEF724F8002211460F20FEF7A8
:1090C0002CF80F20FEF71CF8002211461020FEF7A6
:1090D00024F81020FEF714F8002211461120FEF7A4
:1090E0001CF81120FEF70CF8002211463A20FEF77A
:1090F00014F83A20FEF704F8002211463B20FEF750
:109100000CF83B20FDF7FCFF08BD000000100240FA
:1091100000B585B000BF6C48806940F040006A49E6
:1091200088610846806900F04000009000BF00BFE1
:1091300000BF0846806940F01000886108468069D9
:1091400000F01000009000BF00BF00BF084680691B
:1091500040F0040088610846806900F00400009037
:1091600000BF00BF00BF0846806940F0080088616A
:109170000846806900F00800009000BF00BF00BFF3
:109180000846806940F0200088610846806900F048
:109190002000009000BF00BF012249F255514B480A
:1091A000FDF712FF012241F295314948FDF70CFF0E
:1091B000012241F601114748FDF706FF00228021F8
:1091C0004248FDF701FF01224EF280114248FDF7AF
:1091D000FBFE01224AF2AA514048FDF7F5FE0022AB
:1091E0004FF480413D48FDF7EFFE49F2D550019024
:1091F000012002900220049001A93448FDF738FDB7
:1092000046F62A200190002002900120039001A937
:109210002E48FDF72DFD42F20A0001900020029039
:109220000120039001A92A48FDF722FD41F2953063
:109230000190012002900320049001A92448FDF729
:1092400017FD41F6011001900120029003200490C7
:1092500001A92048FDF70CFD032001900020029099
:10926000039001A91C48FDF703FD4FF491500190B4
:10927000002002900120039001A91748FDF7F8FC97
:109280004EF280100190012002900320049001A969
:109290001148FDF7EDFC4EF2AA500190012002901A
:1092A0000220049001A90D48FDF7E2FC40F655208C
:1092B0000190002002900120039001A90748FDF7CA
:1092C000D7FC05B000BD00000010024000180140AE
:1092D0000010014000080140000C01400014014052
:1092E00000B58DB022482349086000204860002165
:1092F00020488160C16001618161FEF702FC18B104
:1093000042211DA002F01EFA4FF48050099009A9D5
:109310001848FEF74FFC18B1482117A002F012FAC6
:109320001448FEF718FE18B14D2113A002F00AFAF6
:1093300000200790089007A90E48FEF7B1FB18B16E
:1093400054210DA002F0FEF900200090019002903F
:109350000490002269460748FEF7C2FD18B15D215E
:1093600005A002F0EFF90348FEF78AFD0DB000BD3D
:1093700000080040780100202E2E2F5372632F74B6
:10938000696D2E630000000000B595B03448354982
:1093900008604720486000213248816040F69F7194
:1093A000C16000210161416180218161FEF7A9FB5B
:1093B00018B174212CA002F0C5F94FF4805011901F
:1093C00011A92848FEF7F6FB18B17A2126A002F071
:1093D000B9F92448FEF75EFE18B17F2122A002F001
:1093E000B1F920200F90002010900FA91D48FEF722
:1093F00057FB18B186211CA002F0A4F96020089048
:109400004FF4FA60099002200A9000200B900C9013
:109410004FF480700D9000200E90002208A9114892
:10942000FEF7B4FD18B192210FA002F08BF90020D5
:10943000019002900390049005904FF40050069024
:109440000020079001A90748FEF7EBFA18B19E210A
:1094500005A002F077F90348FEF712FD15B000BD34
:1094600000340140B80100202E2E2F5372632F7458
:10947000696D2E630000000010B50C480C490860AF
:109480004FF496404860002109488160C160016145
:109490000C21416100218161C161FEF72BFF18B1F0
:1094A000D32104A002F04EF910BD0000004C004092
:1094B0006C0600202E2E2F5372632F757361727409
:1094C0002E63000010B50C480C4908604FF496401C
:1094D0004860002109488160C16001610C2141613F
:1094E00000218161C161FEF705FF18B1E62104A0EA
:1094F00002F028F910BD000000380140AC06002041
:109500002E2E2F5372632F75736172742E630000B9
:1095100010B50C480C4908604FF416504860002103
:1095200009488160C16001610C21416100218161B4
:10953000C161FEF7DFFE18B1F92104A002F002F9C3
:1095400010BD000000440040EC0600202E2E2F53DA
:1095500072632F75736172742E63000010B50C482E
:109560000C4908604FF4966048600021094881600A
:10957000C16001610C21416100218161C161FEF77F
:10958000B9FE20B14FF4867103A002F0DBF810BDE4
:10959000004800402C0700202E2E2F5372632F7599
:1095A000736172742E63000000BFFEE710B50446BD
:1095B000E1884CF60602881A91424BD01EDC4CF62C
:1095C0000202A1EB0200914264D010DC6FF4314042
:1095D000084458B3B0F5985F48D06FF498510844E8
:1095E000002847D0A0F2FF3000285FD14EE00128CC
:1095F00028D002281ED0032858D11FE040F2FC6278
:10960000811A90423ED008DC02281FD0A0F2FC5004
:10961000002847D0FF2849D130E0B1F5877F3DD001
:10962000A1F6FF21D1B1022940D11BE02046F9F774
:1096300015FF41E02046FBF723FE3DE02046FBF707
:109640001FFE39E02046FCF7FFF835E02046FBF727
:10965000F7F831E02046FBF73FFC2DE0204600F014
:109660003FFC29E02046FBF7B5FA25E02046FAF753
:109670003BFF21E02046FAF711FD1DE02046FAF7F6
:1096800067FB19E02046FAF7B9FA15E02046FBF728
:109690008FFD11E02046FBF727FD0DE0204600F08E
:1096A000DBFE09E02046FAF703FC05E048F204017E
:1096B0002046E26B904700BF00BF10BD10B50E48BA
:1096C000007800F00400A8B10B48007820F00400F6
:1096D0000949087009480068401C084908600846A4
:1096E000007800F0010028B10549E720FCF703FEEF
:1096F0000449086010BD0000440000205400002010
:109700001C0100202C00002010B50948007800F052
:10971000010060B10648007820F00100044908709B
:109720000448007C00F0030008B9FFF7D9F810BD29
:10973000440000208C09002010B52A48007800F071
:10974000100000284CD02748007820F01000254950
:10975000087025480068401C234908602348C07AE7
:1097600098B122484068401C204948600846807AE9
:10977000401C88720846807A3C2190FBF1F201FB84
:10978000120010B91948F7F771FE1948007810B1A6
:109790001748FAF765F81748016817480068F6F7A0
:1097A00017FD154908601048007800F0030098B9CB
:1097B0004FF0814110480068F6F794FD0E490860AB
:1097C0000E4890F82F0020B10C490B480068F7F7BD
:1097D000F9FC00200849086001210948FDF7F0FB69
:1097E00010BD00004400002058000020D4090020D3
:1097F000BC0900202C0000205C0000202C0100206F
:109800000008014010B53148007800F0020000283F
:109810005BD02E48007820F002002C49087000F040
:109820003FF902F0F7FAFCF7FBFB2948007A68B130
:10983000F7F7E0FE0020264908722648007828B194
:109840002448F8F7CBF80020224908702248007A13
:1098500008B1F7F73DFF1E48007858B11C48007862
:10986000401E1B4908700846807818B10846807869
:10987000401E88701948007828B118480078401EAA
:109880001649087000BF1448007868B11248007883
:10989000401E114908700846007828B91048808D8C
:1098A00040F400500E4988850B48407820B10A48A2
:1098B0004078401E0849487001F0F8FA00F044F87A
:1098C000FCF762FD0748F7F771F810BD440000206F
:1098D000F8010020440A0020900500202205002005
:1098E0006A0F00202C0E002010B50748007800F009
:1098F000800040B10448007820F0800002490870E0
:10990000FCF710FD00BF10BD4400002070470000B0
:1099100002480068C0F30220704700000CED00E030
:1099200010B5002807DA0A07140E054A00F00F03E5
:109930001B1FD45403E00A07130E024A135410BD30
:1099400018ED00E000E400E01F4800681F490860CF
:109950001F48007804280EDB1E48007800F0400005
:1099600048B11948006800F4003020B1084600688A
:1099700020F4803008601648407804280FDB154832
:10998000007800F0800050B10F48006800F400300B
:1099900028B90E48006820F480300C4908600C4853
:1099A000807904280FDB0B48008800F4804050B118
:1099B0000548008800F4004028B90448006820F4F5
:1099C0008040024908607047080000200C00002019
:1099D0008C0900200400002070470000D721114AA4
:1099E0001170002151709170002006E000220D4995
:1099F000091D21F81020411CC8B20528F6DBE7211B
:109A0000094A1170002151709170002006E0002277
:109A10000549091D21F81020411CC8B20528F6DBB4
:109A2000704700000E0100201C01002008B5084905
:109A30000968C9084FF47A72B1FBF2F14143009111
:109A400000BF00BF00994A1E00920029F9D108BD4D
:109A500094000020704710B5002305E004880C80B6
:109A6000891C801C5C1CA3B29342F7DB10BD000074
:109A700070B506463046F6F701FD44B2601C44B2AC
:109A80003C2C01DD3C2402E0002C00DA00240248DA
:109A900050F82450284670BDD4C10008704700001B
:109AA00010B54FF40071F848FDF782FAF749F84A0B
:109AB000127888540846007849780844F349897830
:109AC0000844022806DBF348006820F00100F14951
:109AD000086005E0EF48006840F00100ED490860CB
:109AE0004FF40061E848FDF763FAEB49E84A127861
:109AF00088540846007849780844E749897808443A
:109B0000022806DBE348006820F00200E149086013
:109B100005E0E048006840F00200DE4908604FF4CC
:109B20008041D948FDF744FADC49D94A1278885473
:109B30000846007849780844D849897808440228BA
:109B400006DBD448006820F00400D249086005E034
:109B5000D048006840F00400CE4908604FF400513E
:109B6000C948FDF725FACE49C94A127888540846F3
:109B7000007849780844CA4989780844022806DBF5
:109B8000C448006820F00800C249086005E0C148E8
:109B9000006840F00800BF4908604FF40071C148F8
:109BA000FDF706FAC049BA4A127888540846007888
:109BB00049780844BC4989780844022806DBB5483E
:109BC000006820F01000B349086005E0B148006863
:109BD00040F01000AF4908604FF40061B148FDF754
:109BE000E7F9B249AA4A12788854084600784978B9
:109BF0000844AE4989780844022806DBA548006875
:109C000020F02000A349086005E0A248006840F069
:109C10002000A04908600121A248FDF7C9F9A44924
:109C20009B4A127888540846007849780844A0492D
:109C300089780844022806DB9648006820F0400036
:109C40009449086005E09348006840F0400091495D
:109C5000086004219348FDF7ABF996498C4A1278C5
:109C6000885408460078497808449249897808441D
:109C7000022806DB8748006820F0800085490860DC
:109C800005E08448006840F08000824908601021A7
:109C90008448FDF78DF988497D4A12788854084632
:109CA000007849780844844989780844022806DB0A
:109CB0007848006820F480707649086005E07548AF
:109CC000006840F480707349086040217548FDF7D2
:109CD0006FF97A496E4A12788854084600784978B4
:109CE0000844764989780844022806DB69480068F8
:109CF00020F400706749086005E06648006840F499
:109D000000706449086020216D48FDF751F96D49E4
:109D10005F4A1278885408460078497808446949AF
:109D200089780844022806DB5A48006820F48060DD
:109D30005849086005E05748006840F4806055497C
:109D400008604FF400715E48FDF732F95E49504AF1
:109D50001278885408460078497808445A49897826
:109D60000844022806DB4B48006820F4006049499B
:109D7000086005E04748006840F400604549086015
:109D800002214148FDF714F95049414A127888549C
:109D900008460078497808444C49897808440228E4
:109DA00006DB3C48006820F480503A49086005E032
:109DB0003848006840F4805036490860082132482D
:109DC000FDF7F6F84249324A12788854084600787E
:109DD000497808443E4989780844022806DB2D4822
:109DE000006820F400502B49086005E0294800680D
:109DF00040F400502749086002213648FDF7D8F8A2
:109E00003549234A1278885408460078497808442E
:109E1000314989780844022806DB1E48006820F48E
:109E200080301C49086005E01A48006840F4803022
:109E30001849086008212748FDF7BAF82749144A4D
:109E4000127888540846007849780844234989786C
:109E50000844022806DB0F48006820F400300D4952
:109E6000086005E00B48006840F4003009490860CC
:109E700007480078401C0649087008460078032807
:109E800001DB0020087010BD0018014060000020B8
:109E900090000020040000206300002066000020E5
:109EA00069000020001401406C0000206F000020B9
:109EB0007200002075000020780000207B00002048
:109EC000000C01407E000020810000208400002062
:109ED00087000020001001408A0000208D00002033
:109EE00070B504466089372873D018DC1E2871D0FD
:109EF0000CDC0A2875D004DC012828D005286BD199
:109F000056E0142869D01928F9D199E023287CD08B
:109F100028287BD02D287AD03228F0D14AE1552844
:109F200076D008DC3C2874D0412873D0462872D003
:109F30005028E4D190E15A286ED05F286DD0642873
:109F40006CD0A0F57F40F0380028D8D10AE2FD4857
:109F500090F82C0000F0010080B1FB480068000C74
:109F600020F00401F848006861F31240F6490860E7
:109F700048F20C012046E26B904705E2F348007876
:109F80000A2810DAF0480068000C20F00401EE48BE
:109F9000006861F31240EC49086048F292012046E3
:109FA000E26B9047F0E10020606114206081EBE1FA
:109FB000E748007800F0080080B1002211464CF616
:109FC0000200F6F795FC6071607948B10A20608163
:109FD00006E0FDE056E004E0CCE126E014206081DC
:109FE000D2E16179DB4850F8210040894FF6FF71DA
:109FF000884219D16179D74850F82100C08970B9D9
:10A0000014206081002060610EE055E065E0C4E04E
:10A010002AE1E5E0EFE014E131E163E179E148F2C2
:10A0200042012046E26B9047AEE16069401C6061EE
:10A030006069642803D91920608100206061A3E170
:10A04000C5484089B0F5805F10DAC3484089C349EC
:10A0500009688883002211464CF60100F6F748FC97
:10A060006071607910B11E2060818DE16069401CD3
:10A0700060616069C82804D948F20C012046E26B8F
:10A08000904781E16179B34850F8210040894FF64B
:10A09000FF7188420FD16179AE4850F82100C08924
:10A0A00020B9232060810020606104E048F2420171
:10A0B0002046E26B904767E1A948006840F0100035
:10A0C000A74908606069401C60616069642803D921
:10A0D000002060612820608156E19F484089B0F5EA
:10A0E000806F16DA9D480068808BB0F5406F10DDF8
:10A0F0009948408900F5805098490968898B401A31
:10A1000000B29549C8800846C088404200B2C88065
:10A1100040E091484089B0F5406F11DD8F480068FC
:10A12000808BB0F5806F0BDA8C480068808B00F56F
:10A13000805089494989401A00B28749C88029E07E
:10A140008548408985490968898B88420EDD8248A7
:10A15000408982490968898B401A00B27E49C880CB
:10A160000846C088404200B2C88013E07A4840895F
:10A170007A490968898B884209DA78480068808BB7
:10A1800075494989401A00B27349C88002E000202D
:10A190007149C8802D206081F6E04FF420706E492F
:10A1A000488200210120FAF715FB0120E0613720E9
:10A1B0006081E9E04FF42070674948820021012066
:10A1C000FAF708FB37206081E069401CE061DBE0C2
:10A1D0006148407818B9002060613C206081D3E07C
:10A1E0006069401C60616069642803D90020606177
:10A1F00041206081C8E058484089B0F5805F1FDA8F
:10A20000554840895449C988084405B2002D03DAED
:10A2100005F5805005B205E0B5F5805F02DBA5F5D8
:10A22000805005B24D48E26900681C3020F8125099
:10A23000E069132802D34620608101E0322060816A
:10A24000A2E04FF420704449488200210120FAF72F
:10A25000C1FA5020608197E03F48407818B900204B
:10A260006061552060818FE06069401C60616069B9
:10A27000642803D9002060615A20608184E0364858
:10A280004089B0F5805F2CDA334840893249C9886B
:10A29000084405B2002D03DA05F5805005B205E04B
:10A2A000B5F5805F02DBA5F5805005B2A9B22B4A57
:10A2B0001268908BF9F772F8032802DA5F20608148
:10A2C0000FE021480068000C20F004011E480068DF
:10A2D00061F312401C49086048F242012046E26BDB
:10A2E000904751E0F7F71AF910B9642060810FE048
:10A2F00015480068000C20F004011348006861F361
:10A3000012401149086048F242012046E26B904732
:10A310003AE001F005FF064626B131462046E26BE1
:10A32000904702E02046A16B884707480068000C70
:10A3300020F004010448006861F3124002490860FB
:10A3400022E000006A0F0020480000208C09002055
:10A350000C000020400F0020F80000200CCA00086C
:10A36000080000202046A16B884700210846FAF724
:10A3700031FA09E048F204012046E26B90470021DF
:10A380000846FAF727FA00BF00BF70BD10B5F7F70F
:10A3900019F9084808490968C163042200F13C0121
:10A3A0000648FEF713FA062002494870C8200870D4
:10A3B00010BD000090050020E8C500082C07002013
:10A3C00010B5F7F70BF908480849D1F80510C16333
:10A3D000042200F13C010648FEF7F8F90620024984
:10A3E0004870C820087010BD90050020E8C500081E
:10A3F0002C07002038B505464FF6FF7000EA4504EB
:10A40000A01D1249C880552081F89A01AA210F4841
:10A4100080F89B1180F89C41211280F89D11201D2D
:10A4200081B20B4800F06CFA00909DF801200848BA
:10A43000211D42549DF80020611D42540348C288EA
:10A4400003490448FEF7C2F938BD0000F8010020B6
:10A4500092030020AC06002070B5044660892828CD
:10A4600072D008DC012812D00A2833D0142874D006
:10A470001E286BD19CE0322869D03C2868D0462841
:10A4800067D0A0F57F40F0380028F2D1A9E1002084
:10A490006061DE498869DE49F6F76EF805D20A2068
:10A4A0006081DA48FEF77CFC04E01E206081D7481A
:10A4B000FEF776FC0020E061A061D448FEF770FC56
:10A4C000D448006840F48050D24908600020D24946
:10A4D000088399E16069401C6061606914283BD37E
:10A4E00000206061CC48008B401CCB490883088B5E
:10A4F000C11700EB91718910A0EB810159B9C548D2
:10A50000006840F48050C34908605A22BF49C348DC
:10A510000068F6F7FFFEBD498869C0490968F8F789
:10A5200027FF05B2052D15DAA069401CA061A069BE
:10A530000A2811D900206061E061A06114206081C7
:10A540000020B549088307E06DE006E050E1A5E092
:10A55000DFE01BE10020A06156E16069401C606102
:10A560006069142823D300206061AB48008B401C35
:10A57000A9490883088BC11700EB91718910A0EBE2
:10A58000810159B9A348006840F48050A14908608E
:10A590005A229E49A1480068F6F7BCFE9E48008BEF
:10A5A0009A49896A884202D32046A16B88472BE1E9
:10A5B0006069401C60616069142833D300206061C9
:10A5C0009548008B401C94490883088BC11700EB09
:10A5D00091718910A0EB810149B98E48006840F45F
:10A5E00080508C4908603220884981F82D008749C5
:10A5F00088698A490968F8F7BBFE05B23C2D0FDA75
:10A60000A069401CA061A06905280BD900206061E9
:10A61000E061A0612820608100207F49088301E07B
:10A620000020A061F0E06069401C6061606914284E
:10A6300033D3002060617848008B401C7649088342
:10A64000088BC11700EB91718910A0EB810149B90A
:10A650007048006840F480506E49086014206B49CF
:10A6600081F82D00694988696C490968F8F780FE0E
:10A6700005B21E2D0FDAA069401CA061A069052853
:10A680000BD900206061E061A06132206081002070
:10A690006149088301E00020A061B5E06069401CC9
:10A6A00060616069142833D3002060615A48008BD0
:10A6B000401C59490883088BC11700EB9171891020
:10A6C000A0EB810149B95348006840F480505149DA
:10A6D00008600F204D4981F82D004C4988694F4989
:10A6E0000968F8F745FE05B20A2D0FDAA069401C8B
:10A6F000A061A06905280BD900206061E061A0611C
:10A700003C20608100204449088301E00020A061D2
:10A710007AE06069401C60616069142835D30020CC
:10A7200060613D48008B401C3B490883088BC11782
:10A7300000EB91718910A0EB810159B9354800688F
:10A7400040F48050334908600F2230493348006894
:10A75000F6F7E0FD2D49886930490968F8F708FEE9
:10A7600005B2052D0FDAA069401CA061A06905287B
:10A770000BD900206061E061A0614620608100206B
:10A780002549088301E00020A0613DE06069401C8C
:10A7900060616069142823D3002060611E48008B2B
:10A7A000401C1D490883088BC11700EB917189106B
:10A7B000A0EB810159B91748006840F48050154951
:10A7C00008600F22114915480068F6F7A3FD1248EA
:10A7D000008B0E49896A884202D32046A16B8847C4
:10A7E00012E000200C4908832046A16B88470BE04B
:10A7F00048F204012046E26B90470648006820F4C6
:10A8000080500449086000BF00BF70BD2C010020CB
:10A8100000004743080000206A0F00202C000020A1
:10A8200010B501200949087009480A4948630846DB
:10A83000416B88470820074981F8300006480749DE
:10A84000C860001D8860001D486010BDBC09002064
:10A85000198D00082C010020AC0F00200C0A0020EC
:10A8600042898281C1814FF6FF724281C288028192
:10A87000C26A1278521CC36A1A70704710B5012060
:10A880001349087002201349087003201249087008
:10A890000420124908700E48FEF70AFA0D48FEF728
:10A8A00007FA0D48FEF704FA0C48FEF701FA0848CB
:10A8B0000B49486501460A4881650649C165064954
:10A8C0000166064941660420054981F8500010BD23
:10A8D0006C0D0020AC0D0020EC0D00202C0E002093
:10A8E000EC0E00204FF6FF714181C18801810021EB
:10A8F000C1818181C16A0978491CC26A117070479F
:10A9000070B502460C46FF25FF2309E012F8010B43
:10A9100080EA05010648405C80EA03050548435C7F
:10A92000201EA4F10106B4B2F0D143EA052070BDA7
:10A93000F2C50008F2C6000810B5FCF75FFBFDF792
:10A940006AF84048008840B13E480088401E3D49B2
:10A95000088080213C48FCF733FB3C480068401CE1
:10A960003A490860084600680A2869D30020086050
:10A970003748007840F001003549087035480069D3
:10A98000401C34490861084600690521B0FBF1F21A
:10A9900001FB1200002853D12D48007840F002003E
:10A9A0002B4908702B484069401C2A4948610846D9
:10A9B00000690A21B0FBF1F201FB1200F0BB244850
:10A9C000007840F0040022490870224800693221D2
:10A9D000B0FBF1F201FB120080BB1D48007840F093
:10A9E00008001B4908701B4800696421B0FBF1F2A4
:10A9F00001FB120010BB1648007840F0100014490B
:10AA0000087014480069C821B0FBF1F201FB120084
:10AA100028B90F48007840F020000D4908700D4813
:10AA200000694FF4FA71B0FBF1F201FB120028B992
:10AA30000748007840F08000054900E000E0087019
:10AA400010BD00001E00002000180140180000206A
:10AA5000440000208C09002010B596B001200C9015
:10AA600000040D9000200E90012010900220139001
:10AA7000C10314914FF4E01115910CA8FCF77CFD73
:10AA800020B140F20B111CA000F05CFE0F200790DB
:10AA900002200890002009904FF480600A90002066
:10AAA0000B90022107A8FCF723FC20B140F21911FA
:10AAB00011A000F047FE102001900020069001A890
:10AAC000FCF77EFB20B14FF490710BA000F03AFE32
:10AAD000FCF7E0FC4FF47A71B0FBF1F42046FCF790
:10AAE00080FF0420FCF768FF00221146501EFCF78F
:10AAF00014FB16B010BD00002E2E2F5372632F6D65
:10AB000061696E2E630000001148006840F001008A
:10AB10000F490860084640680E4908400C494860E3
:10AB2000084600680C490840094908600846006862
:10AB300020F4802008600846406820F4FE00486049
:10AB40004FF41F008860C803044908607047000084
:10AB5000001002400000FFF8FFFFF6FE08ED00E0E5
:10AB600010B50E48FDF7C0F80D488078A0B90C4824
:10AB7000808A401C00B20A4988820846B0F9141045
:10AB8000B0F91200401E814206DB002004494870E3
:10AB900000210248FDF7C0FA10BD0000B8010020F6
:10ABA000F8000020002202681F4B98420ED01F4B75
:10ABB00098420BD0B0F1804F08D01D4B984205D081
:10ABC0001C4B984202D01C4B984203D122F07002D9
:10ABD0004B681A43144B98420ED0144B98420BD03A
:10ABE000B0F1804F08D0124B984205D0114B9842DB
:10ABF00002D0114B984203D122F44072CB681A4321
:10AC000022F080024B691A4302608B68C3620B68B2
:10AC10008362054B984202D0044B984201D10B69E4
:10AC20000363012343617047002C0140003401405D
:10AC30000004004000080040000C004030B5002334
:10AC4000012404FA01F3046A9C430462046A02FAD0
:10AC500001F52C43046230BD30B50C4600218168FB
:10AC600021F47F4142EA032525432943816030BD19
:10AC70000A460021816821F0700142F00703194360
:10AC80008160704730B5002400220023056A25F05A
:10AC900001050562026A4368846924F0700424F0A7
:10ACA00003040D682C4322F002028D682A43114DE3
:10ACB000A84200D103E0104DA84206D100BF22F007
:10ACC0000802CD682A4322F004020A4DA84202D0AD
:10ACD000094DA84207D123F4807323F400734D6912
:10ACE0002B438D692B43436084614D684563026249
:10ACF00030BD0000002C01400034014030B500247C
:10AD000000220023056A25F010050562026A4368E7
:10AD1000846924F4E04424F440740D6844EA052472
:10AD200022F020028D6842EA0512124DA84200D19D
:10AD300003E0114DA84207D100BF22F08002CD6888
:10AD400042EA051222F040020A4DA84202D00A4D02
:10AD5000A84209D123F4806323F400634D6943EAD8
:10AD600085038D6943EA8503436084614D6885638B
:10AD7000026230BD002C01400034014030B5002497
:10AD800000220023056A25F480750562026A436883
:10AD9000C46924F0700424F003040D682C4322F4E9
:10ADA00000728D6842EA0522124DA84200D103E0EC
:10ADB000114DA84207D100BF22F40062CD6842EADB
:10ADC000052222F480620B4DA84202D00A4DA8420F
:10ADD00009D123F4805323F400534D6943EA05134A
:10ADE0008D6943EA05134360C4614D68C56302621F
:10ADF00030BD0000002C01400034014030B500227D
:10AE000000230024056A25F480550562036A44681E
:10AE1000C26922F4E04222F440720D6842EA05223F
:10AE200023F400538D6843EA0533084DA84202D04D
:10AE3000074DA84204D124F480444D6944EA8514A6
:10AE40004460C2614D680564036230BD002C01405E
:10AE50000034014030B50B46144600210022026A3E
:10AE6000056A25F001050562816921F0F00141EADA
:10AE7000041122F00A021A438161026230BD30B52A
:10AE80000B46144600210022056A25F010050562D4
:10AE90008169026A21F4704141EA043122F0A00282
:10AEA00042EA03128161026230BD000010B50E4813
:10AEB00040894FF6FF71884202D00B48FEF776FBBF
:10AEC0000A4840894FF6FF71884202D00748FEF7D2
:10AED0006DFB074840894FF6FF71884202D0044855
:10AEE000FEF764FB10BD00006C0D0020AC0D0020CF
:10AEF000EC0D0020144840894FF6FF71884203D0C2
:10AF00004FF6F07010494881104840894FF6FF71A4
:10AF1000884203D04FF6F0700C4948810C484089B4
:10AF20004FF6FF71884203D04FF6F0700849488110
:10AF3000084840894FF6FF71884203D04FF6F07001
:10AF400004494881704700006C0D0020AC0D0020C2
:10AF5000EC0D00202C0E0020012806D002280FD076
:10AF6000032818D004282CD120E01C4949894FF629
:10AF7000FF72914203D04FF6F071184A51812BE0D5
:10AF8000174949894FF6FF72914203D04FF6F0718D
:10AF9000134A518120E0134949894FF6FF729142CB
:10AFA00003D04FF6F0710F4A518115E00E494989DF
:10AFB0004FF6FF72914203D04FF6F0710A4A518169
:10AFC0000AE0064949894FF6FF72914203D04FF6D5
:10AFD000F071024A518100BF00BF70476C0D002024
:10AFE000AC0D0020EC0D00202C0E00200146214865
:10AFF000C08888420BD11F4840894FF6FF729042AB
:10B0000005D04FF6F0701B4A5081012070471A4856
:10B01000C08888420BD1184840894FF6FF72904291
:10B0200005D04FF6F070144A50810220EEE7134825
:10B03000C08888420BD1114840894FF6FF72904278
:10B0400005D04FF6F0700D4A50810320DEE70C4822
:10B05000C08888420BD10A4840894FF6FF7290425F
:10B0600005D04FF6F070064A50810420CEE700204C
:10B07000CCE700006C0D0020AC0D0020EC0D002092
:10B080002C0E002010B50248FDF78EF810BD000010
:10B090006C06002070B505466C6A0020E085E084EF
:10B0A0002046FDF77FF870BD70B506460025746A2E
:10B0B00020684069C0F3C01594F83900212805D1F3
:10B0C00025B10020E084204600F082F82068406925
:10B0D000C0F3801594F83A00222805D125B100204C
:10B0E000E085204600F054F8E06B40F01000E0638B
:10B0F0002046FDF757F870BD70B505466C6A2868A4
:10B10000006800F02000B0B90020E0852068C06829
:10B1100020F480702168C8602068406920F0010038
:10B12000216848612068406920F04000216848613A
:10B13000202084F83A002046FDF746FB70BD70B52C
:10B140000446656A2846FDF740FB70BD70B50546AC
:10B150006C6A2868006800F0200070B90020E08464
:10B160002068406920F08000216848612068C0683C
:10B1700040F040002168C86002E02046FDF774FB03
:10B1800070BD70B50446656A2846FDF7A5FB70BD25
:10B190000168C96821F490710268D1600168496949
:10B1A00021F0010102685161202180F83A107047B6
:10B1B00010B504462068C06820F040002168C860CF
:10B1C000202084F839002046FDF74EFB002010BDFA
:10B1D0000168C96821F0C0010268D160202180F8AF
:10B1E0003910704770B5044694F83A0022284AD1C5
:10B1F000A068B0F5805F13D1A56A206940B92068C6
:10B200004068C0F308002880A06A801CA06219E092
:10B2100020684068C0B22880A06A401CA06211E08B
:10B22000206938B920684068C1B2A26A501CA06287
:10B23000117007E02068406800F07F01A26A501C8E
:10B24000A0621170E08D401E80B2E085C8B9206810
:10B25000C06820F020002168C8602068C06820F421
:10B2600080702168C8602068406920F00100216872
:10B270004861202084F83A002046FDF7A5FA002016
:10B2800070BD0020FCE70220FAE700002DE9F04144
:10B29000044600252068006920F44050E168084316
:10B2A000216808612169A068084361690843054372
:10B2B0002068C06841F20C61884328432168C86057
:10B2C0002068406920F44070A16908432168486102
:10B2D0005F49206888425CD1FCF7F2F800EBC001BE
:10B2E00001EB001061688900B0FBF1F6FCF7E8F8AB
:10B2F00000EBC00101EB001061688900B0FBF1F0C8
:10B300006421B0FBF1F000EBC00101EB0010A6EBF3
:10B310008000322101EB00106421B0FBF1F000F05D
:10B32000F006FCF7CDF800EBC00101EB00106168FE
:10B330008900B0FBF1F06421B0FBF1F006EB0016E0
:10B34000FCF7BEF800EBC00101EB0010616889005A
:10B35000B0FBF1F7FCF7B4F800EBC00101EB001013
:10B3600061688900B0FBF1F06421B0FBF1F000EB03
:10B37000C00101EB0010A7EB8000322101EB0010AF
:10B380006421B0FBF1F000F00F00304421688860C8
:10B390005BE0FCF785F800EBC00101EB0010616891
:10B3A0008900B0FBF1F6FCF77BF800EBC00101EB84
:10B3B000001061688900B0FBF1F06421B0FBF1F08E
:10B3C00000EBC00101EB0010A6EB8000322101EB85
:10B3D00000106421B0FBF1F000F0F006FCF760F81B
:10B3E00000EBC00101EB001061688900B0FBF1F0D7
:10B3F0006421B0FBF1F006EB0016FCF751F800EB0E
:10B40000C00101EB001061688900B0FBF1F7FCF7A7
:10B4100047F800EBC00101EB001061688900B0FB48
:10B42000F1F06421B0FBF1F000EBC00101EB001082
:10B43000A7EB8000322101EB00106421B0FBF1F09A
:10B4400000F00F00304421688860BDE8F081000002
:10B4500000380140014691F8390021282CD1886834
:10B46000B0F5805F0FD10A6A1088C0F308000B683E
:10B470005860086918B9086A801C086209E0086AFF
:10B48000401C086205E00B6A581C086218780B68BB
:10B490005860C88C401E80B2C88458B90868C0681B
:10B4A00020F080000B68D8600868C06840F0400059
:10B4B0000B68D860002070470220FCE710B50348F5
:10B4C000FCF772FE00F018F810BD0000AC0600207A
:10B4D00010B500F04FF80248FCF766FE10BD000002
:10B4E000EC06002010B500F07FF80248FCF75CFE87
:10B4F00010BD00002C07002008B51B48006800683C
:10B50000C0F3001070B300BF002000901648006820
:10B5100000680090144800684068009000BF00BFB9
:10B52000124800684068C0F5C870114988800F480B
:10B53000006800684FF6FE7108400C490968086011
:10B540004FF4C870094909684860084800680068F5
:10B5500040F00100054909680860012004490872AB
:10B560005020087008BD0000AC060020F407002041
:10B57000F801002008B5194800680068C0F3001001
:10B5800058B300BF00200090144800680068009085
:10B59000124800684068009000BF00BF1048006873
:10B5A0004068C0F132000F4988800D48006800688B
:10B5B0004FF6FE7108400A490968086032200849C0
:10B5C0000968486006480068006840F001000449C6
:10B5D0000968086001200349087208BDEC060020D4
:10B5E0007C0800202205002008B519480068006882
:10B5F000C0F3001050B300BF002000901448006852
:10B6000000680090124800684068009000BF00BFCA
:10B61000104800684068C0F132000F49888001205E
:10B6200008720C48006800684FF6FE71084009492E
:10B6300009680860322007490968486005480068C1
:10B64000006840F0010003490968086008BD000077
:10B650002C070020480900209005002010B54FF469
:10B66000C8721E491E48FDF74DF81D480068C068A5
:10B6700040F010001A490968C8600120FBF718FA69
:10B68000322218491848FDF73DF817480068C0688D
:10B6900040F0100014490968C8600120FBF708FA5F
:10B6A000322212491248FDF72DF811480068C0688F
:10B6B00040F010000E490968C8600120FBF7F8F956
:10B6C00008480A38F6F77CF908480A38F6F778F996
:10B6D000012004490A39087210BD0000020200204E
:10B6E000AC0600202C050020EC0600209A05002066
:10B6F0002C07002000BFFEE7002004498861486253
:10B70000C86188620862C862704700008C09002026
:10B710002DE9F04104460E461746FBF793FA002543
:10B720000AE036F815C06246002321460120FBF7E7
:10B7300031FAA41C681C85B2BD42F2DBFBF720FA8B
:10B74000BDE8F08100BFFEE70FB4084B10B504A9B7
:10B7500002AA039800F01CF8044602A9002000F099
:10B7600048FA204610BC5DF814FB0000F3BB00084B
:10B7700002E008C8121F08C1002AFAD170477047BA
:10B78000002001E001C1121F002AFBD17047000018
:10B790002DE9FF4F8DB00F460546002606E025280F
:10B7A0000BD0DDE90F1290476D1C761C287800281D
:10B7B000F5D111B03046BDE8F08F0024A246A14675
:10B7C0000122EC4900E0044315F8013F203B02FA56
:10B7D00003F00842F7D128782A2810D06FF02F0202
:10B7E0002878A0F13001092914D80AEB8A0102EB6C
:10B7F000410144F0020400EB010A6D1CF0E701CFA7
:10B800005FEA000A03D544F40054CAF1000A44F088
:10B8100002046D1C28782E2817D115F8010F44F06A
:10B8200004042A280ED06FF02F022878A0F13001EE
:10B8300009290AD809EB890102EB410100EB010952
:10B840006D1CF2E757F8049B6D1C28786C280FD00C
:10B8500006DC4C2817D068280DD06A2814D104E0E3
:10B86000742810D07A280FD10DE044F400140AE0B7
:10B8700044F4801401E044F440146978814202D118
:10B8800004F580146D1C6D1C2A786E2A1FD00CDC08
:10B89000632A31D004DC002A8BD0582A11D1A3E0CE
:10B8A000642A68D0692A0CD165E0732A2ED004DCA2
:10B8B0006F2A73D0702A04D19BE0752A6FD0782A42
:10B8C0006ED01046DDE90F129047761C50E1C4F3AC
:10B8D0000250022806D0032809D0042801CF09D03D
:10B8E000066045E101CFF117C0E9006140E101CFF9
:10B8F00006803DE106703BE117F8040B8DF800006F
:10B9000000208DF80100EB46012003E057F804BB4E
:10B910004FF0FF3061074FF0000102D40DE008F155
:10B920000101884649450FDA8045F8DB1BF808100D
:10B930000029F4D108E008F1010188468142FADBD0
:10B940001BF808100029F6D1DDE90F23AAEB080047
:10B950008146214600F036F9304400EB080604E049
:10B96000DDE90F121BF8010B9047B8F10108F7D27F
:10B9700021464846F7E00A21C4F302534FF0000B7A
:10B980000891022B04D001CFC117032B09D00AE084
:10B99000FF1D27F00707F7E8020108E032E01FE08B
:10B9A00020E000B2C117042B01D140B2C117031E21
:10B9B00071F1000307DA4FF0000CD0EB0C006CEBD8
:10B9C00001012D2302E0230504D52B238DF824301B
:10B9D000012303E0E30701D02023F7E7984658E06E
:10B9E0000A2110E010210EE010204FF0000B08900B
:10B9F0000CE010214FF0000B44F004044FF0080954
:10BA0000089103E008214FF0000B0891C4F30253A2
:10BA1000022B04D001CF0021032B06D006E0FF1D2E
:10BA200027F00707F7E8020103E080B2042B00D1FA
:10BA3000C0B24FF0000823072BD5702A07D0DDF8DD
:10BA400020C08CF0100C5CEA0B0C05D00EE04023FB
:10BA50008DF82430012308E050EA010306D030239A
:10BA60008DF824308DF8252002239846DDF820C07B
:10BA70008CF0080C5CEA0B0C0BD150EA010301D1ED
:10BA8000630706D530238DF824304FF00108A9F163
:10BA90000109582A04D038A20B9208AA0A920BE096
:10BAA0003AA2F9E75B46089AF4F770FD0B9B9B5CA2
:10BAB0000A9A521E0A92137050EA0102F2D10A98B1
:10BAC000ADEB000000F1200B600702D524F48034B8
:10BAD00001E04FF00109D94502DDA9EB0B0000E0C0
:10BAE000002000EB0B0141440890AAEB010AE0039F
:10BAF00006D4DDE90F232146504600F063F80644E2
:10BB00004FF0000908E009A911F80900DDE90F125A
:10BB1000904709F10109761CC145F4DBE0030CD51F
:10BB2000DDE90F232146504600F04CF8064404E0BE
:10BB3000DDE90F1230209047761C0899481E0890C6
:10BB40000029F5DC08E00A980A990078491C0A9156
:10BB5000DDE90F129047761CBBF10001ABF1010B40
:10BB6000F1DC21465046DDE90F2300F019F80644C8
:10BB70006D1C1BE60928010030313233343536376D
:10BB80003839616263646566000000003031323329
:10BB900034353637383941424344454600000000C9
:10BBA0002DE9F041044600251E461746880404D4BA
:10BBB00005E039462020B0476D1C641EF9D52846A3
:10BBC000BDE8F0812DE9F041044600251E4690466F
:10BBD000C80301D5302700E02027880404D505E0FC
:10BBE00041463846B0476D1C641EF9D52846BDE86D
:10BBF000F0810A68531C0B60107070472DE9F0410A
:10BC000005460027B84600241CE0601C142190FB68
:10BC1000F1F201FB120805F11C0030F81400B0F538
:10BC2000805F00DB7F1C05F11C0232F8181032F82F
:10BC30001400F7F78FFB0646C82E01DBD22E00DD7D
:10BC40007F1C641C142CE0DB47B10848808D40F059
:10BC50004000064988850120BDE8F0810348808DB9
:10BC600020F04000014988850020F5E76A0F002098
:10BC700010B5002821D0114B0022001F196803E0E5
:10BC8000814203D80A4649680029F9D152B11368A4
:10BC9000841A9C4204D1006818441060104602E0E7
:10BCA000506000E0186039B102680B1A934203D16A
:10BCB0000B681A4402604968416010BD980000207A
:10BCC0002DE9FE4F83460E460196019E700000F05E
:10BCD000AFF90446002504E03BF8150024F81500F0
:10BCE0006D1CB542F8D3002518E0002711E034F8A8
:10BCF0001710781C34F81000814209DD34F817A0C1
:10BD0000781C34F8100024F81700781C24F810A0D0
:10BD10007F1CB01E401BB842E9D86D1CB01EA84263
:10BD2000E3D8701E34F810002188401AB0F5006F77
:10BD30000CDA701E34F810002188401A80B200908E
:10BD40002046FFF795FF0098BDE8FE8F4FF00008F2
:10BD500000250BE034F81500B0F5006F05DA34F873
:10BD60001500404501DD34F815806D1CB542F1D356
:10BD70004FF4805900250BE034F81500B0F5006F42
:10BD800005DD34F81500484501DD34F815906D1CCB
:10BD9000B542F1D349464046F7F7DCFA82462046E1
:10BDA000CDF808A0FFF764FF0298CDE770B5002535
:10BDB000002417E0FEF7EAFA00201549A1F8400038
:10BDC00040F2DC50FAF774FE1148B0F8400000F47D
:10BDD000807008B1681C45B24FF49670FAF768FE9F
:10BDE000601C44B2032CE5DB012D01DD00240DE0D5
:10BDF00001240748808D40F4005005498885084695
:10BE0000408D48F22601084301494885204670BD0F
:10BE10006A0F002010B5FAF775F80446B4F5805F94
:10BE200006DB5448808D40F080005249888505E04B
:10BE30005048808D20F080004E4988854D48848789
:10BE4000808F4D4948814B49888FF7F783FE4A49D7
:10BE5000C870484890F82C0000F04000F0B1084647
:10BE6000408900280FDD0846408903280BDC0120AB
:10BE700008704248C079FF280FDA4048C079401C5A
:10BE80003E49C87109E03C48C07840F080003A491A
:10BE9000C870002008703949C87110BD3648C07894
:10BEA00000F0800058B9334890F82C0000F00100F1
:10BEB00028B9304890F82C0000F0800050B12E488E
:10BEC000C07840F080002C49C870002008702B49D1
:10BED000C8710BE00120284908702848C079FF2864
:10BEE00004DA2648C079401C2449C8712248C07829
:10BEF0002049C887224800780A2190FBF1F201FB13
:10BF00001200204921F810401D480078401C1C49AF
:10BF100008700A211B48FFF7D3FE0446154890F825
:10BF20002C0000F00100D0B9124890F82C0000F06D
:10BF30008000A0B91048407888B9032C0FDC124863
:10BF4000006820F00050104908600C48007AFF2873
:10BF50000EDA0A48007A401C0849087208E00A48CC
:10BF6000006840F00050084908600020034908724A
:10BF700000BF92E76A0F0020F80000208C09002023
:10BF8000100000206401002004000020FBF73EF8B0
:10BF9000FEF762FDFDF7BCF8FDF75AF8FDF7A0F9D2
:10BFA000FDF76AFAFDF78EFAFDF7B2FAFDF7D6FA59
:10BFB000FDF7EAF9FFF7A0FBFEF732FC1A4800682C
:10BFC00040F48000184908604FF48000F4F792FFB5
:10BFD0000020F4F7CBFF4FF49670FAF769FDFEF7F7
:10BFE0004DFC1248FAF75CF9FFF738FBFDF7F6FC59
:10BFF0004FF49670FAF75CFD40F6B830FAF758FD4A
:10C00000FFF7D4FE4FF49670FAF752FD00F046F8B1
:10C0100009E0FDF779FBFDF7F5FBFDF74FFBFDF7B9
:10C020008BFBFDF761FCF4E7080000205C0F0020AB
:10C03000F0B50B30154D20F007010024144A0FE035
:10C0400003688B420BD38B4205D95E1A43184768AD
:10C05000C3E9006700E04368136002C004E0021D0A
:10C0600010680028ECD12046002802D1286808B1C9
:10C070000020F0BD064A07481060074A121A22F055
:10C080000702C0E9002401202860D7E79C000020B7
:10C0900098000020841000208012002030B59DB050
:10C0A000052400BF372201A91A48FDF7D4FC6C21F2
:10C0B00001A8FEF725FC0546BDF87000A84201D195
:10C0C000002411E0641E032C0ED21348808D40F42E
:10C0D0008070114988850846808D40F04000888531
:10C0E00048F228001DB030BD002CDBD101A8FFF7BD
:10C0F00085FD40B10848808D40F0400006498885A4
:10C1000048F20A00EEE76E2201A90448F4F73CF871
:10C110000020E7E700E007086A0F0020CE0F0020AC
:10C1200070B59CB06C212848FEF7EAFB27490968E6
:10C13000A1F86C00052400BF2548F7F727FC4FF451
:10C14000FA70F7F7F7F92249C8312148F5F7D8F91D
:10C1500006460EB9002406E0641E032C03D248F202
:10C1600029001CB070BD002CE6D1052400BF372289
:10C1700015491748FFF7CCFA4FF4FA70F7F7DAF9D8
:10C18000372269461248FDF766FC6C216846FEF7C7
:10C19000B7FB05460D480068B0F86C00A84209D10D
:10C1A000BDF86C0009490968B1F86C10884201D1EA
:10C1B000002405E0641E032C02D248F22800D0E7D8
:10C1C000002CD4D10020CCE7CE0F00200CCA0008F0
:10C1D00000E007080000000077BE1F3DC1CAA13D76
:10C1E00046B6F33DC1CA213E83C04A3E46B6733EC1
:10C1F000F2D28D3ED34DA23EB4C8B63E9643CB3E5E
:10C2000077BEDF3E5839F43E1D5A043F8D970E3FEE
:10C21000FED4183F6F12233FDF4F2D3FD9CE373F5B
:10C220004A0C423FBA494C3F2B87563F2506613F97
:10C2300096436B3F8FC2753F0000803F7D3F853F37
:10C24000355E8A3FB29D8F3F6ABC943FE7FB993FC2
:10C25000643B9F3FE17AA43F9A99A93F17D9AE3F2B
:10C260009318B43F1058B93F8D97BE3F46B6C33FB1
:10C27000C3F5C83F3F35CE3FBC74D33F39B4D83F38
:10C28000B6F3DD3FF853E33F7593E83FF2D2ED3F5D
:10C290006F12F33FEC51F83F6891FD3F7368014026
:10C2A0009318044052B806401058094031080C4019
:10C2B000F0A70E40AE471140CFF713408D971640C0
:10C2C0004C3719406DE71B402B871E404C372140EF
:10C2D0000AD72340C9762640E9262940A8C62B4024
:10C2E000C9762E4087163140A8C633406666364070
:10C2F0008716394046B63B4000003840250641408D
:10C3000046B64340666646402506494046B64B4021
:10C3100004564E4025065140E3A55340045656406E
:10C32000C3F55840E3A55B40A2455E40C3F56040BD
:10C3300081956340A245664060E5684081956B4009
:10C340003F356E4060E570401F8573403F35764055
:10C35000FED478401F857B40DD247E404E628040C5
:10C360005EBA81400000C842CDCCCF427B94D74218
:10C370000A57DF427B14E742CDCCEE42E17AF64227
:10C38000F628FE4266E60243C3B506438F820A439F
:10C390003D4A0E43EC1112437BD415437B94194361
:10C3A0007B541D43CD0C21431FC52443E17A284310
:10C3B000852B2C4329DC2F43AE873343A4303743EE
:10C3C0000AD73A4352783E439A194243C3B545438C
:10C3D0005C4F494366E64C43E17A5043CD0C5443ED
:10C3E000000000009643CB3EBA494C3FE7FB993F23
:10C3F0003F35CE3F736801406DE71B4066663640AF
:10C400002506514081956B403D0A8340894190400B
:10C4100073689D40C976AA40BC74B7404E62C44060
:10C420007D3FD1404A0CDE40E5D0EA408195F7409F
:10C43000273102418D9708410C020F41BC74154110
:10C4400085EB1B417F6A2241C3F5284106812F41BC
:10C450009318364121B03C41DF4F4341CFF749416A
:10C46000BE9F5041C74B5741E7FB5D4108AC64415B
:10C470005A646B41AC1C7241FED4784181957F4176
:10C48000F6288341448B864191ED8941DF4F8D41F0
:10C4900039B49041A01A9441068197416DE79A41C1
:10C4A000D34D9E4146B6A141B81EA5412B87A84158
:10C4B000AAF1AB411D5AAF419CC4B2410E2DB64109
:10C4C0008195B941F4FDBC416666C041D9CEC341F6
:10C4D0004C37C741B29DCA410C02CE417368D1416D
:10C4E000C1CAD4410E2DD8415C8FDB419EEFDE41A5
:10C4F000D34DE24108ACE5412506E9414260EC41FB
:10C5000052B8EF416210F3415A64F64146B6F94120
:10C510003108FD41022B0042ECD10142C9760342B1
:10C52000A61B054277BE0642486108420C020A4239
:10C53000D1A20B4289410D423BDF0E42E77B104204
:10C540009318124233B31342CD4C154260E51642A4
:10C55000EE7C184275131A42F6A81B42713D1D422B
:10C56000DFCF1E424E622042B6F32142198423429D
:10C5700075132542C5A02642142E28425EBA2942D0
:10C580009C442B42D9CE2C420A572E423BDF2F42ED
:10C59000606531427FEA3242986E3442AAF13542F8
:10C5A000B6733742B6F33842B0723A42A4F03B4217
:10C5B0008B6C3D426DE73E424861404217D9414293
:10C5C000DF4F43429CC4444252384642FCA9474292
:10C5D000A01A494231884A42C3F54B4242604D425B
:10C5E000BAC94E422D325042D3490D8A00DA490D64
:10C5F0008A0000C1814001C0804101C0804100C16A
:10C60000814001C0804100C1814000C1814001C022
:10C61000804101C0804100C1814000C1814001C012
:10C62000804100C1814001C0804101C0804100C102
:10C63000814001C0804100C1814000C1814001C0F2
:10C64000804100C1814001C0804101C0804100C1E2
:10C65000814000C1814001C0804101C0804100C1D2
:10C66000814001C0804100C1814000C1814001C0C2
:10C67000804101C0804100C1814000C1814001C0B2
:10C68000804100C1814001C0804101C0804100C1A2
:10C69000814000C1814001C0804101C0804100C192
:10C6A000814001C0804100C1814000C1814001C082
:10C6B000804100C1814001C0804101C0804100C172
:10C6C000814001C0804100C1814000C1814001C062
:10C6D000804101C0804100C1814000C1814001C052
:10C6E000804100C1814001C0804101C0804100C142
:10C6F000814000C0C101C30302C2C60607C705C509
:10C70000C404CC0C0DCD0FCFCE0E0ACACB0BC90979
:10C7100008C8D81819D91BDBDA1A1EDEDF1FDD1D89
:10C720001CDC14D4D515D71716D6D21213D311D1B9
:10C73000D010F03031F133F3F23236F6F737F53509
:10C7400034F43CFCFD3DFF3F3EFEFA3A3BFB39F939
:10C75000F83828E8E929EB2B2AEAEE2E2FEF2DED09
:10C76000EC2CE42425E527E7E62622E2E323E12179
:10C7700020E0A06061A163A3A26266A6A767A56589
:10C7800064A46CACAD6DAF6F6EAEAA6A6BAB69A9F9
:10C79000A86878B8B979BB7B7ABABE7E7FBF7DBD09
:10C7A000BC7CB47475B577B7B67672B2B373B17139
:10C7B00070B0509091519353529296565797559509
:10C7C00094549C5C5D9D5F9F9E5E5A9A9B5B9959B9
:10C7D0005898884849894B8B8A4A4E8E8F4F8D4D89
:10C7E0004C8C4484854587474686824243834181F9
:10C7F0008040AA100000000C1801460255034E04A8
:10C8000043050006000700080009010A000B000CA0
:10C8100000AA100000000C18010002000300040030
:10C82000050006000700080009010A000B010C02C0
:10C83000AA100000000C180100020003000400050B
:10C840000006000700080009010A000B020C10AAEC
:10C85000100000000C18013802380338043805387D
:10C8600006380738083809010AFF0BFF0CFF2020A3
:10C870005445535420200052455F544553542000E2
:10C880005445535453544F500020204441544520A4
:10C890002000444154412053504100455252202031
:10C8A000535041005345454B484F4C45004F56456A
:10C8B0004E53544F50004F56454E48454154004248
:10C8C000205244204F46460042205244204F4E20E2
:10C8D000002042205245414420002042205A455227
:10C8E0004F200042205057204F46460042205057CC
:10C8F00020204F4E0050554D50204F464600505579
:10C900004D5020204F4E0046414E20204F464600BD
:10C9100046414E2020204F4E004E325620204F469A
:10C9200046004E32562020204F4E004449534B20A3
:10C93000525354004E455854484F4C4500444953B7
:10C940004B5455524E004449534B465245450044C2
:10C9500049534B20205550004449534B444F574EA8
:10C96000004C4944434C4F5345004C4944204F50E0
:10C97000454E00414952434C4F53450041495220D6
:10C980004F50454E002041444A55535420004348DF
:10C9900045434B494E4700434845434B204F4B00CE
:10C9A00050555420204355500020574549474820B2
:10C9B0002000205245445543452000494E435245EE
:10C9C0004153450057414954434F4F4C004D4F563A
:10C9D00045204C49440050555420204C49440020E7
:10C9E00053414D504C45200057414954374D494E15
:10C9F00000574149542042414E002020202045202C
:10CA00002020002020204C3144202000CE0F002088
:10CA1000800F00200000000000000000010203045D
:10CA20000607080900000000010203044CCA0008C0
:10CA300000000020A000000070B70008ECCA000849
:10CA4000A0000020E015000080B7000800000000F2
:10CA500000000000000000000000000000000000D6
:10CA600000000000000000000000000000000000C6
:10CA700000000000000000000000A0410000A041F4
:10CA80000000A04100007042000000000000000013
:10CA90000000000000000000000000000000000096
:10CAA0000000000000000000000000000000000086
:10CAB0000000000000000000000000000000000076
:10CAC0000000000000000000000000000000000066
:10CAD0000000000000000000000000000000000056
:0CCAE00000A24A0400000000000000005A
:0400000508000131BD
:00000001FF
